:1010010002A78702849F900B327402F0E59620E7D5
:10101100FB759601759701E4900B42F0A37403F000
:10102100A3F0220291667814E6FF22028905900A54
:10103100497401F0A37409F0A37415F0900A48747F
:101041000AF022027D9A90087EEBF0A3EAF0A3E970
:10105100F0A3ECF0A3EDF0A3E07002A3E07002C1F5
:101061000F900881E0FEA3E0FF7C007D08129EF056
:1010710090087EE0FBA3E0FAA3E02FF9EA3EFA90A4
:10108100088AEBF0A3EAF0A3E9F0900888E0FEA358
:10109100E0FF7C007D08129EF0900885E0FBA3E054
:1010A100FAA3E02FF9EA3EFA90088DEBF0A3EAF0FB
:1010B100A3E9F0900881E0FEA3E0FF7C007D081227
:1010C1009EF0900890ECF0A3EDF0900888E0FEA36C
:1010D100E0FF7C007D08129EF0900892ECF0A3EDF9
:1010E100F0900890E0FEA3E0FF6D7002EE6C6002EC
:1010F10041ECEF4E7002410E90088AE0FBA3E475CB
:10110100F001129F3CA9F0FA129E3CFF900892E078
:10111100FCA3E0FD244EF582740B3CF583E05F9067
:101121000898F0C374089DFFE49CFEC3900884E016
:101131009FEE6480F8900883E064809890088DE0C9
:10114100FB403CA3E0FAA3E0F9129E3CFF90089219
:10115100A3E02445F582740B3CF583E05F129E7792
:10116100900892E0FEA3E0FFC374089FFFE49EFE97
:10117100C3900884E09FF0900883E09EF08072A302
:10118100E0FAA3E0F9129E3CFF900883E0FCA3E0A3
:10119100FD900892E0F8A3E02DFDE83CFC744F2D92
:1011A100F582740B3CF583E0FE900892E0FCA3E02D
:1011B1002445F582740B3CF583E04E5F129E7790D7
:1011C1000898E0FF900883E0FCA3E0FD900893E01D
:1011D1002DFD900892E03CFC74452DF582740B3C8A
:1011E100F583E0FEEF5E900898F0E4900883F0A3A9
:1011F100F090088DE0FBA3E475F001129F3CA9F08B
:10120100FA129E3CFF900898E04F129E7790088357
:10121100E0FAA3E0FB7C007D08FFAE02129EF09095
:101221000894EEF0A3EFF07C007D08AF03AE02124C
:101231009EF0A3ECF0A3EDF0900894E07002A3E01F
:10124100603F900894E0FEA3E0FF90088DE0FBA3CF
:10125100E0FAA3E0F8AC02AD0390088AE0FBA3E05A
:10126100FAA3E0F9129DF4900894E0FEA3E0FF9048
:10127100088BEE8FF0129F2690088EEE8FF0129F52
:1012810026900896E0FEA3E0FF4E7002C10F900881
:101291008DE0FBA3E0FAA3E0F9129E3CFD744E2F12
:1012A100F582740B3EF583E05D129E7790088DE028
:1012B100FBA3E0FAA3E0F9C003C002C001129E3C07
:1012C100FF90088AE0FBA3E0FAA3E0F9129E3CFE3E
:1012D100900896E0FCA3E02445F582740B3CF5836D
:1012E100E05E4FD001D002D003C10C900892E0FE25
:1012F100A3E0FFD3900891E09FEE6480F8900890FE
:10130100E06480984070A3E09FFF900890E09E9079
:101311000894F0A3EFF0900894E0FEA3E0FFC374FB
:10132100089F900897F0E49E900896F090088AE054
:10133100FBA3E475F001129F3CA9F0FA129E3CFD5B
:10134100A807088002C333D8FC90089CF0E0FF9006
:10135100088AE0FBA3E0FAA3E0F9129E3CFE9008A4
:1013610096A3E0FDEEA805088002C313D8FC4FFF49
:1013710090089CF0804A900890E0FEA3E0FFC390A3
:101381000893E09FFF900892E09E900896F0A3EFEB
:10139100F0900896E0FEA3E0FFC374089F900895C3
:1013A100F0E49E900894F090088AE0FBA3E0FAA391
:1013B100E0F9129E3CFDA807088002C313D8FCFF88
:1013C100900892E0FCA3E0244EF582740B3CF58377
:1013D100E05F90089CF0900892E0FEA3E0FFC374E8
:1013E100089FFFE49EFEC3900884E09FEE6480F8AE
:1013F100900883E064809890088DE0FB403EA3E074
:10140100FAA3E0F9129E3CFF900892E0FCA3E024CD
:1014110045F582740B3CF583E05F129E779008924C
:10142100E0FEA3E0FFC374089FFFE49EFEC39008A3
:1014310084E09FF0900883E09EF08072A3E0FAA31D
:10144100E0F9129E3CFF900883E0FCA3E0FD9008C8
:1014510092E0F8A3E02DFDE83CFC744F2DF5827479
:101461000B3CF583E0FE900892E0FCA3E02445F5F7
:1014710082740B3CF583E04E5F129E7790089CE0EE
:10148100FF900883E0FCA3E0FD900893E02DFD9020
:101491000892E03CFC74452DF582740B3CF583E029
:1014A100FEEF5E90089CF0E4900883F0A3F09008B2
:1014B1008DE0FBA3E475F001129F3CA9F0FA129EA6
:1014C1003CFF90089CE04F129E77900883E0FEA3BA
:1014D100E0FF7C007D08129EF0900898EEF0A3EFEB
:1014E100F090089874FFF5F0129F26C364809480F1
:1014F100406590088AE0FBA3E475F001129F3CA9C6
:10150100F0FA129E3CFF900894A3E0FEEFA80608B3
:101511008002C333D8FC90089CF0E0FF90088AE079
:10152100FBA3E0FAA3E0F9129E3CFE900896A3E02B
:10153100FDEEA805088002C313D8FC4FFF90089C5C
:10154100F090088DE0FBA3E475F001129F3CA9F037
:10155100FAEF129E77808A900883E0FEA3E0FF7C79
:10156100007D08129EF090089AECF0A3EDF04C700B
:1015710002C10F90088AE0FBA3E475F001129F3CC1
:10158100A9F0FA129E3CFF900894A3E0FEEFA80692
:10159100088002C333D8FC90089CF0E0FF90088AD1
:1015A100E0FBA3E0FAA3E0F9129E3CFE900896A3AB
:1015B100E0FDEEA805088002C313D8FC4FFF900898
:1015C1009CF090089AE0FCA3E0FD2445F582740BA1
:1015D1003CF583E05F90089CF090088DE0FBA3E070
:1015E100FAA3E0F9129E3CFF744E2DF582740B3C78
:1015F100F583E05F129E7790088DE0FBA3E0FAA3EC
:10160100E0F9129E3CFF90089CE04F129E772290D9
:101611000B77EBF0A3EAF0A3E9F0A3EDF0E0FE54C1
:1016210007900B7CF0EEC394085002E18EE4900B1E
:101631007BF0900B7AE0131313541FFFA3E0C39FB9
:101641004002E18E900B77E0FBA3E0FAA3E0F99072
:101651000B7BE0FF75F008A4F582E92582F9EA35F4
:10166100F0FA129E3C9008CAF0900B77A3E0FAA31F
:10167100E0F975F008EFA42401F582E435F0F58373
:10168100E92582F9EA3583FA129E3C9008CBF09065
:101691000B77A3E0FAA3E0F9900B7BE075F008A4C7
:1016A1002402F582E435F0F583E92582F9EA3583F0
:1016B100FA129E3C9008CCF0900B77A3E0FAA3E0DD
:1016C100F975F008EFA42403F582E435F0F583E918
:1016D1002582F9EA3583FA129E3C9008CDF0900BF1
:1016E10077A3E0FAA3E0F9900B7BE075F008A4245E
:1016F10004F582E435F0F583E92582F9EA3583FAC8
:10170100129E3C9008CEF0900B77A3E0FAA3E0F98B
:1017110075F008EFA42405F582E435F0F583E92599
:1017210082F9EA3583FA129E3C9008CFF0900B774C
:10173100A3E0FAA3E0F9900B7BE075F008A424067E
:10174100F582E435F0F583E92582F9EA3583FA1269
:101751009E3C9008D0F0900B77A3E0FAA3E0F975D6
:10176100F008EFA42407F582E435F0F583E925823A
:10177100F9EA3583FA129E3C9008D1F07BFF7AA8F2
:10178100798E123000900B7BE004F0C133900B7C1A
:10179100E0D39400404B900B7AE0131313541F7560
:1017A100F008A4A3F0900B7AE0FFA3E0FEC39F50E2
:1017B10027900B77E0FBA3E0FAA3E02EF9E43AFAD5
:1017C100129E3C9008CAF07BFF7AA879B7123000CC
:1017D100900B7BE004F080CD7BFF7AA879BD1230BD
:1017E1000022E59620E7FB75960EE4F597E5962035
:1017F100E7FB759611759720900B427404F022E473
:10180100FFFEFDFC90087012A106900870E0F8A39D
:10181100E0F9A3E0FAA3E0FB900A0BE0FFE4FCFD92
:10182100FEEB2FFFEE3AFEED39FDEC38FC9008702F
:1018310012A106900870E0F8A3E0F9A3E0FAA3E092
:10184100FBC000900A0CE0FFE4FCFDFE780812A04A
:10185100F3D000EB2FFFEA3EFEE93DFDE83CFC90B2
:10186100087012A106900870E0F8A3E0F9A3E0FA6D
:10187100A3E0FBC000900A0DE0FFE4FCFDFE781040
:1018810012A0F3D000EB2FFFEA3EFEE93DFDE83C5C
:10189100FC90087012A106900A0AE024FE70022151
:1018A1004524FE7002219F24FC7002416C24F870D3
:1018B1000241C5147002614424F170028128241F81
:1018C1006002A166900870E0FCA3E0FDA3E0FEA326
:1018D100E0FF90088312A1067F16121D9F90086FEA
:1018E100748BF01247EF90086FE0241BF0E0FF12B9
:1018F1006C77900874EFF09008877401F0A3740876
:10190100F0A3746EF07B017A08796DE4FFFE125842
:101911000090086DE0540FC3940E400A90086FE0E8
:101921006480946C40C0129B9590086DE0FE540F4A
:10193100900959F0EEC4540FA3F090086EE090099D
:101941005BF0A16E900870E0FCA3E0FDA3E0FEA3B4
:10195100E0FF90088312A1067F16121D9F7F0112DE
:10196100864512775D90086BEEF0A3EFF012809739
:10197100900869EEF0A3EFF0E4FF12864590086B42
:10198100E0FAA3E0FF900869A3E0C39F900959F032
:10199100EAFD900869E0C39D90095AF0A16E90009C
:1019A1000FE004F0900861E004F090000FE0FBD339
:1019B100943540097435F0E4900959A16B90087091
:1019C100E0FCA3E0FDA3E0FEA3E0FF75F004EBA4BF
:1019D100240CF582E5F03400F58312A106900A0E7D
:1019E100E0FF74E32BF582E43400F583EFF0900A15
:1019F1000FE0900862F0900870E0FCA3E0FDA3E026
:101A0100FEA3E0FF90000BE0F8A3E0F9A3E0FAA346
:101A1100E0FBC312A0CF5014900870E0FCA3E0FDDE
:101A2100A3E0FEA3E0FF90000B12A106900870E076
:101A3100FCA3E0FDA3E0FEA3E0FF90085DE0F8A3B6
:101A4100E0F9A3E0FAA3E0FBD312A0CF4014900881
:101A510070E0FCA3E0FDA3E0FEA3E0FF90085D12AF
:101A6100A10690095974FCF0A3613F90000F740125
:101A7100F0900861F0900870E0FCA3E0FDA3E0FEA7
:101A8100A3E0FF90001012A106900A0EE09000E47E
:101A9100F0900870E0FCA3E0FDA3E0FEA3E0FF905E
:101AA100000B12A106900870E0FCA3E0FDA3E0FE8C
:101AB100A3E0FF90085D12A10690095974FEF0A3FE
:101AC10004F0A16E900A0BE0FF7E00900855EEF045
:101AD100A3EFF0FD900A0CE0FFED900855CFF0A3C5
:101AE100EFF0900A0DE0FF900824EEF0A3EFF0FD77
:101AF100900A0EE0FFED900824CFF0A3EFF0900ADA
:101B01000FE0FF900846EEF0A3EFF0FD900A10E021
:101B1100FFED900846CFF0A3EFF090095974FEF065
:101B2100C3900825E09432900824E09400500CE41E
:101B3100F0A37432F090095974FFF090095A74FFC0
:101B4100F0A16EE4FFFEFDFC90087412A10674FF83
:101B5100FFFEFDFC90087812A10690095974FEF071
:101B6100A304F0900862E090095BF0900855E0FC56
:101B7100A3E090095CF0ECA3F0900824E0FCA3E062
:101B810090095EF0ECA3F0900846E0FCA3E0900918
:101B910060F0ECA3F090085DE0FCA3E0FDA3E0FEA3
:101BA100A3E0FF900962EFF090085DA3A3A3E078A2
:101BB1000812A0E0900963EFF090085DE0FCA3E05B
:101BC100FDA3E0FEA3E0FF781012A0E0900964EF0E
:101BD100F090000BE0FCA3E0FDA3E0FEA3E0FF908A
:101BE1000965EFF090000BA3A3A3E0780812A0E031
:101BF100900966EFF090000BE0FCA3E0FDA3E0FE8E
:101C0100A3E0FF781012A0E0900967EFF09008615F
:101C1100E0900968F09000E4E0900969F090000F0D
:101C2100E090096AF0A16E900A0FE0FE900A0EE0C2
:101C3100FDEDFF900874EEF0A3EFF07F07129744DB
:101C4100900876EFF07F08129744900877EFF0E460
:101C5100FD7F07129916E4FD7F081299169008700E
:101C6100E0FCA3E0FDA3E0FEA3E0FF90088312A146
:101C7100067F16121D9F9009577442F0A37440F01D
:101C8100900A5EE0FBA3E0FAA3E02401F9E43AFA4A
:101C9100129E3C900A5DF0A37401F0A37409F0A3B5
:101CA1007457F090095974FEF0A304F01298BC9097
:101CB1000874E0FEA3E0FFD394E8EE9403401BEF29
:101CC1002420FFE43EFEEF7806CEC313CE13D8F9ED
:101CD100FF7C007D30129E89801A900874E0FEA37B
:101CE100E0FF7C007D30129E89EF7806CEC313CED3
:101CF10013D8F9FF90084BEEF0A3EFF0E490084EF3
:101D0100F07F011286457F017E001287DF129A0A59
:101D1100129CC67F8F129A75900A10E0B4010512C9
:101D2100840F80057F9E129A757D0A7C007F807EDC
:101D3100001291BAE4F50EF50F1299BBEF6006128D
:101D41001027EF60CEE4FF128645900876E0FD7F14
:101D510007129916900877E0FD7F081299169008EE
:101D6100547401F02290095974FFF0A3F0900957BF
:101D71007442F0A37440F0900A5EE0FBA3E0FAA382
:101D8100E02401F9E43AFA129E3C900A5DF0A37452
:101D910001F0A37409F0A37457F01298BC229008C3
:101DA10082EFF0A3E0FCA3E0FDA3E0FEA3E0FF903F
:101DB1000B0212A106E4FF12974490088AEFF05437
:101DC100FEFDE4FF129916900882E0641670757B9F
:101DD100017A0879877D037F161293EE900889E0D6
:101DE100547024F0602024D0602724F0602E24F069
:101DF100603524F0603C2470704390088B7401F0CE
:101E0100A374F4F0803E90088BE4F0A374FAF080A0
:101E11003390088BE4F0A374C8F0802890088BE419
:101E2100F0A37464F0801D90088BE4F0A37432F089
:101E3100801290088BE4F0A37419F08007E49008F5
:101E41008BF0A3F090088BE0FEA3E0FBAA06E4F977
:101E5100F8900883E0FCA3E0FDA3E0FEA3E0FF12FD
:101E6100A02790089312A106900893E0FCA3E0FD3F
:101E7100A3E0FEA3E0FF780612A0E0EE543FFE903F
:101E8100088DEEF0A3EFF090088DE0FCA3E0FDAE2D
:101E9100047806C333CE33CED8F92DFFEC3EFE9045
:101EA100088FF0A3EFF0E4FCFD900893E0F8A3E0C5
:101EB100F9A3E0FAA3E0FBD312A0CF401C90089055
:101EC100E02441F090088FE03400F090088EE004A7
:101ED100F0700690088DE004F0900893A3A3E0FE53
:101EE100A3E0FFC3900890E09FF090088FE09EF080
:101EF10090088DE0FEA3E0FBAA06C3900890E09451
:101F01002190088FE09400401C90088EE024FFF09F
:101F110090088DE034FFF0900890E024DFF0900805
:101F21008FE034FFF0C3900890E0942090088FE098
:101F310094004011EB1B70011AA3E024E0F090081B
:101F41008FE034FFF090088FE0FEA3E0FFC3942000
:101F5100EE940050A5EF9410EE94004010E024E0C0
:101F6100F090088FE034FFF0EB1B70011A90088F9E
:101F7100E0FEA3E0FFC390088EE09FFF90088DE094
:101F81009E900891F0A3EFF0900890E02BFF90084D
:101F91008FE03AAD07FC900882E064167047EDAE21
:101FA100047806CEC313CE13D8F9540FFF900889D5
:101FB100E054F04FF0900891E0FAA3E0FBEA5403FB
:101FC100FFAE05EE25E025E054FC4F900888F09027
:101FD1000887EBF07B017A0879879008B77403F0E2
:101FE1007F16128DAE12700090088AE0FDE4FF02A8
:101FF1009916E4900869F0A3F053C97F029ABAE4F4
:10200100900863F0900866F0A374C8F053D9BF122A
:102011001FF3D2AF1296537BFF7AA6798512300057
:102021007F5E7EC67D0D7C0090001012A10690009F
:10203100E474D8F07F527EC87D0D7C0090001412AC
:10204100A1069000E574D8F07F467ECA7D0D7C0024
:1020510090001812A1069000E674D8F07F3A7ECC69
:102061007D0D7C0090001C12A1069000E774D8F051
:102071007F2E7ECE7D0D7C0090002012A106900067
:10208100E874D8F07F227ED07D0D7C009000241270
:10209100A1069000E974D8F07F167ED27D0D7C00F8
:1020A10090002812A1069000EA74D8F07F0A7ED42D
:1020B1007D0D7C0090002C12A1069000EB74D8F0ED
:1020C1007FFE7ED57D0D7C0090003012A106900030
:1020D100EC74D8F07FF27ED77D0D7C009000341235
:1020E100A1069000ED74D8F07FE67ED97D0D7C00CD
:1020F10090003812A1069000EE74D8F07FDA7EDBF2
:102101007D0D7C0090003C12A1069000EF74D8F088
:102111007FCE7EDD7D0D7C0090004012A1069000F7
:10212100F074D8F07FC27EDF7D0D7C0090004412F8
:10213100A1069000F174D8F07FB67EE17D0D7C00A0
:1021410090004812A1069000F274D8F07FAA7EE3B5
:102151007D0D7C0090004C12A1069000F374D8F024
:102161007F9E7EE57D0D7C0090005012A1069000BF
:10217100F474D8F07F927EE77D0D7C0090005412BC
:10218100A1069000F574D8F07F867EE97D0D7C0074
:1021910090005812A1069000F674D8F07F7A7EEB79
:1021A1007D0D7C0090005C12A1069000F774D8F0C0
:1021B1007F6E7EED7D0D7C0090006012A106900087
:1021C100F874D8F07F627EEF7D0D7C009000641280
:1021D100A1069000F974D8F07F567EF17D0D7C0048
:1021E10090006812A1069000FA74D8F07F4A7EF33D
:1021F1007D0D7C0090006C12A1069000FB74D8F05C
:102201007F3E7EF57D0D7C0090007012A10690004E
:10221100FC74D8F07F327EF77D0D7C009000741243
:10222100A1069000FD74D8F07F267EF97D0D7C001B
:1022310090007812A1069000FE74D8F07F1A7EFB00
:102241007D0D7C0090007C12A1069000FF74D8F0F7
:102251007F0E7EFD7D0D7C0090008012A106900115
:102261000074D8F07F027EFF7D0D7C009000841207
:10227100A10690010174D8F07F5C7E797D0C7C0011
:1022810090008812A10690010274D8F07FEA7E02C4
:102291007D0E7C0090008C12A10690010374D8F091
:1022A1007FDE7E047D0E7C0090009012A1069001DD
:1022B1000474D8F07FD27E067D0E7C0090009412CB
:1022C100A10690010574D8F07FC67E087D0E7C00C2
:1022D10090009812A10690010674D8F07FBA7E0A88
:1022E1007D0E7C0090009C12A10690010774D8F02D
:1022F1007FAE7E0C7D0E7C009000A012A1069001A5
:102301000874D8F07FA27E0E7D0E7C009000A4128E
:10231100A10690010974D8F07F967E107D0E7C0095
:102321009000A812A10690010A74D8F07F8A7E124B
:102331007D0E7C009000AC12A10690010B74D8F0C8
:102341007F7E7E147D0E7C009000B012A10690016C
:102351000C74D8F07F727E167D0E7C009000B41252
:10236100A10690010D74D8F07F667E187D0E7C0069
:102371009000B812A10690010E74D8F07F5A7E1A0F
:102381007D0E7C009000BC12A10690010F74D8F064
:102391007F4E7E1C7D0E7C009000C012A106900134
:1023A1001074D8F07F427E1E7D0E7C009000C41216
:1023B100A10690011174D8F07F367E207D0E7C003D
:1023C1009000C812A10690011274D8F07F2A7E22D3
:1023D1007D0E7C009000CC12A10690011374D8F000
:1023E1007F1E7E247D0E7C009000D012A1069001FC
:1023F1001474D8F07F127E267D0E7C009000D412DA
:10240100A10690011574D8F090000F7432F0129764
:10241100077F017E001287DF900010E0FCA3E0FD42
:10242100A3E0FEA3E0FF123800900864EEF0A3EFF2
:10243100F04E60177FE87E031287DF900864A3E007
:10244100FF1267687FE87E031287DF7BFF7AA67938
:10245100CB900864E0FFA3E09008CACFF0A3EFF0AF
:10246100123000129C5C7DAA7F007E1012986212CD
:102471009C1F900866E07002A3E06010900867E07E
:1024810024FFF0900866E034FFF0803B900864E0A0
:102491007002A3E07F0060027F0474C07E5DA80724
:1024A100088005C333CE33CED8F9900867F0EE909B
:1024B1000866F0900868E06006E4F0C2A280089027
:1024C10008687401F0D2A2126A4980A6E59620E755
:1024D100FB75960EE4F597E59620E7FB759691E579
:1024E1009620E7FB9008C6E597F0900B42E0B40513
:1024F10013E59620E7FBE4F596900B39E0F597E4B8
:10250100900B42F09008C6E0FF30E210E59620E71C
:10251100FB759611E4F597900B42F022EF30E41B26
:10252100E59620E7FB759611759708E59620E7FB80
:10253100759611759780E4900B42F0900B42E06024
:1025410002C12A9008C6E020E002C12A7B017A0B71
:1025510079367D087C007F20128F3A900B39E0FE9E
:10256100900B38E07C002400FFEC3EF0A3EFF090EC
:102571000B3BE0FE900B3AE02400FFEC3EF0A3EFB2
:10258100F0900B3DE0FE900B3CE02400FFEC3EF0B0
:10259100A3EFF0900B36E0547F64217035A3E02463
:1025A100FE601B14602224FA600F14601614601D73
:1025B100240A7072129479807012950F806B123711
:1025C100FF8066129B818061124FFE805C124FFF7B
:1025D1008057900B37E0B40C00504B9025E225E07A
:1025E10073A1FAA1FFC127C104C127C109C10EC14D
:1025F10027C113C118C11DC12212752C802B12874E
:102601005A80261285BA802112920E801C12598F8F
:10261100801712888380121286D0800D128CCF8091
:102621000812969180031217E3900B42E064016057
:1026310002C1FA9008C6E030E102C1FAE59620E74E
:10264100FB759691E59620E7FB9008C6E597F0E0CB
:1026510030E40530E002C1FA9008C67402F0C3907C
:102661000B41E09440900B40E09400403C900B33D0
:10267100E0FBA3E0FAA3E0F97D407C007F2012910A
:102681000F900B34E475F040129F26900B41E0242B
:10269100C0F0900B40E034FFF0900B3FE02440F09D
:1026A100900B3EE03400F08024900B40E0FCA3E06E
:1026B100FD900B33E0FBA3E0FAA3E0F97F20129138
:1026C1000F9008C6E04408F0E4900B42F0900B3CF8
:1026D100E0FEA3E0FFA3E0B50611A3E0B5070C906F
:1026E10008C6E04408F0E4900B42F0E59620E7FBD1
:1026F1007596119008C6E0F597900B42E064026070
:1027010002E1DAE59620E7FB759691E59620E7FB75
:102711009008C6E597F0E020E002E1DA7440F0C3EA
:10272100900B41E09440900B40E09400403C900BB2
:1027310033E0FBA3E0FAA3E0F97D407C007F2012A7
:102741008F3A900B34E475F040129F26900B41E0D4
:1027510024C0F0900B40E034FFF0900B3FE02440A8
:10276100F0900B3EE03400F0801C900B40E0FCA3A5
:10277100E0FD900B337F20128F329008C6E04408B1
:10278100F0E4900B42F0900B3CE0FEA3E0FFA3E0ED
:10279100B50611A3E0B5070C9008C6E04408F0E4C3
:1027A100900B42F0900B42E07019900B37E0B409A6
:1027B10012900B33E0FBA3E0FAA3E0F9129E3CFF79
:1027C100129000900B42E064046005E59620E7FB5F
:1027D1007596119008C6E0F5972290086CEBF0A36E
:1027E100EAF0A3E9F0E4FF90086CE0FBA3E0FAA3B0
:1027F100E02FF9E43AFA129E3C60030F80E922903F
:10280100087CEBF0A3EAF0A3E9F0A3E0FBA3E0FA74
:10281100A3E0F9129F52FDACF0AE047803CEC313CE
:10282100CE13D8F9FF900882EEF0A3EFF0ED540734
:10283100A3F0E92407F9E43AFA12A112900885EB12
:10284100F0A3EAF0A3E9F0E4A3F0A3F0A3F0A3F06E
:10285100A3F0A3F0A37429F075088F90087FE0FB23
:10286100A3E0FAA3E0240AF9E43AFA129E3CF5093E
:1028710090087FA3E0FAA3E02402F9E43AFA129F58
:1028810052FDACF0AE047803CEC313CE13D8F99049
:102891000889F0ED54076003E004F07E007F2C7D91
:1028A100007B007A00793012A335900882E0FCA306
:1028B100E0FDEC540FC454F0FBED54F0FFE4C4F818
:1028C10054F0C8EFC4540F484B7830F6E0540FC4AD
:1028D100F8540FC868FF7831A6079008887402F091
:1028E100900884E0601625E0540E440146F69008F5
:1028F10083E004F07006900882E004F0E490088A16
:10290100F0900883E024FEFF900882E034FFFE90FF
:10291100088AE0C39FE49E503390087FE0FBA3E068
:10292100FAA3E02404F9E43AFA12A11290088AE029
:10293100FF29F9E43AFA129E3CFE900888E02F2420
:1029410030F8A60690088AE004F080B590088AE085
:10295100FF900888E02FF0900884E0FF7002413A70
:10296100900888E0FE242FF9C374089FFF74FFA824
:1029710007088002C333D8FC57F7742F2EF8C00024
:10298100E6FE90087CE0FBA3E0FAA3E02425F9E44D
:102991003AFA129E3CFD900884E0FCEDA804088000
:1029A10002C313D8FC4ED000F6900888E0FE243014
:1029B100F8C000E6FD90087CE0FBA3E0FAA3E02468
:1029C10025F9E43AFA129E3CFCA807088002C333B9
:1029D100D8FC4DD000F674302EF8C000E6FF900808
:1029E1007CE0FBA3E0FAA3E02426F9E43AFA129E84
:1029F1003CFE900884E0FDEEA805088002C313D8D0
:102A0100FC4FD000F6900888E02431F8C000E6FFC2
:102A110090087CE0FBA3E0FAA3E02426F9E43AFA6B
:102A2100129E3CFEC374089DFDEEA805088002C3FA
:102A310033D8FC4FD000F6803890087CE0FBA3E04F
:102A4100FAA3E02425F9E43AFA129E3CFF900888A3
:102A5100E0FE2430F8A60790087CE0FBA3E0FAA38F
:102A6100E02426F9E43AFA129E3CFF74312EF8A6CE
:102A710007900888E02402F07F0712974490088CA1
:102A8100EFF090087FE0FBA3E0FAA3E0240BF9E468
:102A91003AFA129E3CFD7F0712991690087FE0FBDF
:102AA100A3E0FAA3E0240BF9E43AFA129E3CB4FF46
:102AB100047D3E80027D3F7F0D129916E4F50EF5EF
:102AC1000F7F8F129A7590087FE0FBA3E0FAA3E0D5
:102AD1002402F9E43AFA129F52FD7F1B12991690D3
:102AE100087FE0FBA3E0FAA3E02402F9E43AFA123A
:102AF1009F52E5F05403FD7F1A1299169008A074B5
:102B01001DF0A3E4F0A37400F0A37430F0900888E2
:102B1100E09008A4F07B007A0079097D01128F9280
:102B21007F807E00129831E4F50EF50F7F8F129AA7
:102B310075E4900888F090087FE0FBA3E0FAA3E039
:102B41002402F9E43AFA129F5245F0700281837F20
:102B51005E7E80129831E50F30E35C90088DA3E032
:102B6100FD7F1B12991690088DE05403FD7F1A1208
:102B710099167F527E001298317F1C129744EF54B0
:102B81000FFFC3940340027F03900885E0FBA3E09D
:102B9100FAA3E0F9128C627F8F129A757D3F7F0D47
:102BA100129916900885E0FBA3E0FAA3E0F9129EC2
:102BB1003C4480FF029E77E50E30E74290088B741B
:102BC10012F0E50E30E73790088BE0FFB4122F903A
:102BD1000885E0FBA3E0FAA3E0F9128C6290088B70
:102BE100E0FFFD900886E48DF0129F26900888E0B2
:102BF1002FF0530E7F7F5E7E8012983180C47F5EFE
:102C01007E00129831E50F541F60207F1C129744FB
:102C1100EF541FFF90087FE0FBA3E0FAA3E0240C30
:102C2100F9E43AFAEF129E777F0822E4F50EF50FE8
:102C31007F1C129744EF541FFF90088BF090088877
:102C4100E0FEFDEF2DFDE433FCA3E0FFFBD3ED9BA4
:102C51007480F86C984006EF9E90088BF090088B7A
:102C6100E0FF900885E0FBA3E0FAA3E0F9128C6293
:102C710090088BE0FF900888E02FF0900889E0240D
:102C8100FEF090088CE0FD7F07129916900888E00D
:102C9100FF90087FE0FBA3E0FAA3E0240CF9E43AFB
:102CA100FAEF129E777D3F7F0D1299167F002290D9
:102CB100087DEBF0A3EAF0A3E9F0A3EDF0E49008BE
:102CC10090F0900887F0A3F0900885F0A3F07FC002
:102CD100FE1298317F5F7E00129831E50F541F601C
:102CE1000890089074FFF0E1BF530F7F90088A7439
:102CF1008FF0A3749DF07B017A08798A7D02129B83
:102D0100277D407F1A1299167D3F7F0D1299167FFC
:102D1100807E001298317F8F129A75E4F50EF50FBF
:102D21007F1BFE129831E50F5417600890089074CC
:102D3100FEF0E1BFE50F20E302E1BF90087DE0FB7B
:102D4100A3E0FAA3E02402F9E43AFA7F01128C62CB
:102D510090087DE0FBA3E0FAA3E02402F9E43AFA4B
:102D6100129E3C54F81313543FFF7E00900883EEEB
:102D7100F0A3EFF0D39420EE94004009900883E48F
:102D8100F0A37420F0900883A3E0FF90087DE0FB9E
:102D9100A3E0FAA3E02424F9E43AFAEF129E779033
:102DA1000884E02404F0900883E03400F0E0FEA3FE
:102DB100E0FF900887EEF0A3EFF07803C333CE3342
:102DC100CED8F9FF900883EEF0A3EFF0900883E0EE
:102DD100FCA3E0FDEC5403444090088AF0EDA3F01D
:102DE100900883E0FEA3E07803CEC313CE13D8F995
:102DF100F0EE900883F07B017A08798A9008B77425
:102E010002F07F1A128DAEE4F50EF50F90087DE009
:102E1100FBA3E0FAA3E02403F9E43AFA90088DEB6E
:102E2100F0A3EAF0A3E9F0900884E024FF805FC3F7
:102E3100900884E09412900883E09400405A7F0641
:102E41007E80129831E50F5407600890089074FD58
:102E5100F0E1BF7F1C129744900882EFF0530E7F80
:102E610090088DE0FBA3E0FAA3E0F97F12128C62D7
:102E7100900886E02412F0900885E03400F0900874
:102E81008EE475F012129F26900884E024EEF090F3
:102E91000883E034FFF08097E4900881F0E50F5457
:102EA1005F7066900882E02403F00000E02403F0E4
:102EB1000000E02403F07F1C129744EF541F900898
:102EC10082F0D39401403690088DE0FBA3E0FAA391
:102ED100E0F97F01128C62900886E004F0700690A0
:102EE1000885E004F090088EE475F001129F2690A9
:102EF1000884E024FFF0900883E034FFF09008811B
:102F0100E004F0E0D394C840947F5F7E00129831D2
:102F1100E50F5415700790088904F08005E49008C6
:102F210089F0E4F50EF50F900880E0FF129A757FA5
:102F31001C129744EF541F900882F06031E0FFFDAE
:102F4100C3900884E09DF0900883E09400F090081D
:102F51008DE0FBA3E0FAA3E0F9128C62900882E015
:102F6100FF900886E02FF0900885E03400F07F8F15
:102F7100129A757F0F12974490087DE0FBA3E0FA47
:102F8100A3E02427F9E43AFAEF129E77900889E04A
:102F910060069008907401F0900888E024FFF0909A
:102FA1000887E034FFF0900885E0FEA3E0FFA3E08E
:102FB1006E7003A3E06F602490089074FCF0E4F558
:102FC1000EF50F90088A748FF0900880E090088BBE
:102FD100F07B017A08798A7D02129B27E4FD7F1A32
:102FE100129916900890E0FF2212629F1298BC90ED
:102FF1000A0A7402F0900959E06003B401EB2290CF
:1030010008C7EBF0A3EAF0A3E9F0E49008F2F0A31B
:10301100F0A3F0A3F0A3F0A3F0A3F0A3F09008FEB7
:10302100F0A3F0A3F0A3F0A3F090090A04F0A374B5
:1030310008F0A374CAF09008C7E0FBA3E0FAA3E08C
:10304100F9129E3C7002813012A13233EB0A308FAB
:103051002533873033AD3133AD3233AD3333AD3416
:1030610033AD3533AD3633AD3733AD3833AD3930BC
:10307100E24430E25530DA5830E26330E26430AF96
:103081006830E26C30E27530E27800003401E4909F
:103091000908F0A3F09008F6E07004A3E064019041
:1030A10008F67007F0A3F07F258110E4619690087F
:1030B100F6E07002A3E06010900909E004F07006E8
:1030C100900908E004F081139008C7E0FBA3E0FA3F
:1030D100A3E0F9129E3CFF8110900900E4F0A304E3
:1030E100F0E49008FAF0A3F0A3F0A3F09008F6E062
:1030F1007004A3E064016002616B90090DF0A37498
:1031010004F0900908E0FEA3E0FF64024E702690EF
:10311100090DF0A37402F090090AE0FBA3E475F035
:1031210001129F3CA9F0FA129E3CFD9008F4E4F0D4
:10313100A3EDF08021EF64014E90090AE0FBA3E4C6
:1031410075F002129F3CA9F0FA129F52FF9008F409
:10315100E5F0F0A3EFF090090DE0FFA3E09008F295
:10316100CFF0A3EFF0D39008F3E094009008F2E0E1
:1031710094005002418990090DA3E01425E025E057
:10318100FD740F7E00A805088005C333CE33CED869
:10319100F9FF9008F4E05EFEA3E05FA80508800552
:1031A100CEC313CE13D8F9FF9008F2E0FCA3E0FDE3
:1031B1002402F58274093CF583EFF074022DF58247
:1031C10074093CF583E0FFC3940A402BEFD3940FBD
:1031D1005025900900E07002A3E07E5760027E371F
:1031E100EE2FFF9008F2E0FCA3E02402F5827409BF
:1031F1003CF583EFF080219008F2E0FEA3E0FF248C
:1032010002F58274093EF583E02430FD74022FF546
:103211008274093EF583EDF09008F2E0FEA3E0240C
:1032210002F58274093EF583E0B4302A9008FAE091
:103231007002A3E070109008FDE004F07026900881
:10324100FCE004F0801E9008FBE004F0701690088A
:10325100FAE004F0800E9008FBE004F0700690089C
:10326100FAE004F09008F5E0C4F8540FC868F09053
:1032710008F4E0C454F048F09008F3E024FFF09023
:1032810008F2E034FFF0216690090DE0FEA3E0FFB3
:103291002403F58274093EF583E4F09008F6F0A367
:1032A100F09008FEE07002A3E070089008FEEEF0D6
:1032B100A3EFF09008FAE0FEA3E0FFC39008FFE05F
:1032C1009F9008FEE09E4070E49008F2F0A3F09019
:1032D10008FAE0FEA3E0FFC39008FFE09FFF90081B
:1032E100FEE09EFEC39008F3E09F9008F2E09E503E
:1032F100157F301293099008F3E004F070D1900823
:10330100F2E004F080C99008FAE0FFA3E09008F22F
:10331100CFF0A3EFF09008F2E0FEA3E0FFD394001A
:10332100EE940040571292FD9008F3E024FFF090D4
:1033310008F2E034FFF080DD9008FAE0FFA3E090AE
:1033410008F2CFF0A3EFF09008F2E0FEA3E0FFD384
:103351009400EE940040251292FD9008F3E024FFC2
:10336100F09008F2E034FFF080DD9008C7E0FBA3A5
:10337100E0FAA3E0F9129E3CFF129309E49008FEE3
:10338100F0A3F0A380519008F6E07004A3E064017B
:1033910070099008F8F0A304F080779008C7E0FB6B
:1033A100A3E0FAA3E0F9129E3CFF80639008F8E0E5
:1033B1007004A3E064019008C77021E0FBA3E0FA68
:1033C100A3E0F9129E3C24D0FEE434FF9008FEF005
:1033D100A3CEF0E49008F8F0A3F08036E0FBA3E080
:1033E100FAA3E0F9129E3CFF80257F0D129309900C
:1033F10008C7E0FBA3E0FAA3E0F9129E3CFF800FAF
:103401009008C7E0FBA3E0FAA3E0F9129E3CFF128B
:1034110093099008C7E0FBA3E0FAA3E02401F9E4D3
:103421003AFA9008C7EBF0A3EAF0A3E9F0013722DA
:1034310090087EEBF0A3EAF0A3E9F0A3EDF0E490AD
:10344100088BF0A3F0A3F0A3F0900891F0A374030C
:10345100F0E4F50EF50F7F8F129A75E4900891F064
:10346100900881E0FF900891E0C39F504D90087E45
:10347100E0FBA3E0FAA3E0F9900891E0FF75F028E2
:10348100A4F582E92582F9EA35F0FAE4F5F0129F14
:103491007DEF75F028A4FF90087EE0FBA3E0FAA37E
:1034A100E02FF9EA35F0FAE92424F9E43AFAE412D2
:1034B1009E77900891E004F080A6E4F50EF50F9058
:1034C100088AE0600F900882E0FBA3E0FAA3E0F92C
:1034D100A3E080077B007A007900E4FD1250007FB1
:1034E1002C7E01129C66E4F50EF50F900886E0FF34
:1034F100128987E490088DF0A3F07F01FEFDFC9016
:103501000886E0F9F812A0F390088FEEF0A3EFF02F
:10351100900881E0FD90088BE0FEA3E0FFC39DEEE3
:1035210094004002C10D7C007D28129E8990087E86
:10353100E0FBA3E0FAA3E02FF9EA3EFA128E6BEF6B
:103541001460142402706790088EE004F0705F909C
:10355100088DE004F08057900885E0FF7E00C006EA
:10356100C00790088BE0FEA3E0FF7C007D28129E3F
:103571008990087EE0FBA3E0FAA3E02FF9EA3EFA86
:10358100E92404F9E43AA801FCAD03900882E0FBC8
:10359100A3E0FAA3E0F9D007D00612A311EF700E51
:1035A10090088CE004F0700690088BE004F090081D
:1035B10090E024FFF090088FE034FFF0E4F50EF581
:1035C1000F900887A3E0FAA3E0F912A1589008939D
:1035D100EFF0900881E0FFC390088CE09F90088B8A
:1035E100E09400501590088FE07002A3E0600B900A
:1035F1000893E060057F99129A7590088FE0700238
:10360100A3E06008900893E06002A111900892E0A5
:1036110014F090088DE07002A3E0607DE47F01FE6C
:10362100FDFC900886E0F9F812A0F3E47B04FAF9B6
:10363100F812A027A804A905AA06AB0790088DE0F7
:10364100FEA3E0FFE4FCFDD312A0CF500A90088650
:10365100E004F07F9A803DE47F01FEFDFC90088646
:10366100E0F9F812A0F3E47B08FAF9F812A027A810
:1036710004A905AA06AB0790088DE0FEA3E0FFE4CC
:10368100FCFDD312A0CF400A900886E014F07F9C85
:1036910080027F9B129A758005E4900892F0900851
:1036A10081E0FFC390088CE09F90088BE09400506C
:1036B10017900892E06011900887A3E0FAA3E0F95F
:1036C10012A158EF600281F490088BE07002A3E030
:1036D1007021900B0DE024FFF0900B0CE034FFF013
:1036E100E07002A3E07015FF128645129C2D124472
:1036F100AE8000900B0CE4F0A3740AF090088BE00C
:10370100FEA3E0FF229008A6EBF0A3EAF0A3E9F004
:10371100A3EDF0E4FFA3E0FBA3E0FAA3E0F9129E1E
:103721003CFE9008A6E0FBA3E0FAA3E02402F9E442
:103731003AFAEE129E779008AAE0FBA3E0FAA3E022
:103741002401F9E43AFA129E3CFE9008A6E0FBA39C
:10375100E0FAA3E02403F9E43AFAEE129E77900826
:10376100A9E0FEEFC39E50329008ADE0FBA3E0FA62
:10377100A3E02FF9E43AFA129E3CFE9008A6E0FB82
:10378100A3E0FAA3E02404F9E43AFAEF7C0029F972
:10379100EC3AFAEE129E770F80C49008A9E0FF90F0
:1037A10008A6E0FBA3E0FAA3E02424F9E43AFAEF47
:1037B100129E779008B0E0FBA3E0FAA3E0F9129E15
:1037C1003CFF9008A6E0FBA3E0FAA3E02425F9E47E
:1037D1003AFAEF129E779008B0E0FBA3E0FAA3E07B
:1037E1002401F9E43AFA129E3CFF9008A6E0FBA3FB
:1037F100E0FAA3E02426F9E43AFAEF029E77229058
:10380100086912A10690086D7455F0A374AAF0E43A
:10381100A3F0A374FFF07B017A08796D9008B77467
:1038210004F07F16128DAE7E007F047D007B017A4D
:1038310008796D12A3357B017A08796D7D047F16B5
:103841001293EE90086DE0FFB4550EA3E0B4AA09FF
:10385100A3E07005A3E0F460257BFF7AA37988904B
:1038610008CAEFF090086EE09008CBF090086FE086
:103871009008CCF0900870E09008CDF02152C2A1E0
:103881007F017E001287DFD2A17F0C7E001287DFCD
:103891007B017A08796D7D047F161293EE90086D95
:1038A100E06455600FA3E064AA6009A3E06005A38A
:1038B100E0B4FF087BFF7AA379A82152E4F50EF565
:1038C1000F7D207F0D1299167D027F1E1299167FA2
:1038D1008F129A757F92129A757B017A08796D9091
:1038E10008B77404F07F1F128DAE7B017A08796DE1
:1038F1009008B77404F07F1F128DAE7B017A0879AE
:103901006D9008B77404F07F1F128DAE7B017A08A9
:10391100796D9008B77404F07F1F128DAE7B017A28
:1039210008796D9008B77404F07F1F128DAE7B018A
:103931007A08796D9008B77404F07F1F128DAE7FFD
:10394100207E00129831E50F20E50E7BFF7AA379E6
:10395100B71230007E007F0122E4F50EF50F129CB4
:103961002D7F84129A75129CCCEF24C8601C24E828
:10397100602614602324FC601F24257023E4900A30
:10398100F2F07BFF7AA379DB8024900AF27401F0D4
:103991007BFF7AA379F18016900AF27402F0801607
:1039A100129CCC9008CAEFF07BFF7AA47907123001
:1039B100007E007F0F227D02E4FF1299167D067FB3
:1039C100011299167DF07F021299167D0C7F0A1261
:1039D100991690086F7460F090086E74D8F0900892
:1039E1006D744FF07B017A08796D9008B77403F01C
:1039F1007F16128DAE7D027F0B12991690086D74A1
:103A010001F07403F0A3745DF0A37420F07B017ADC
:103A110008796D9008B77403F07F15128DAE7F0B96
:103A210012974490086DEFF04460F0FD7F0B1299FE
:103A3100167D377F0D12991690086D7403F0A374EB
:103A410084F0A3740AF07A08796D128DA4E49008C9
:103A51006DF0A3F0A3F07B017A08796D9008B7743B
:103A610003F07F12128DAEE4FF129776900869E0A1
:103A7100FCA3E0FDA3E0FEA3E0FF90088312A106F2
:103A81007F16121D9F7FB4126C777F147E00128700
:103A9100DF7F0E12974490086DEFF020E0057E0065
:103AA1007F022290086DE020E1057E007F0322E481
:103AB100FEFF22900B70EEF0A3EFF0A3EBF0A3EA70
:103AC100F0A3E9F0E4FFA3F0A3F0FEFD900B71E099
:103AD10024F0900B70E034D8C364809480400FA32D
:103AE100E024F0F0900B70E034D8F00F80DE900B02
:103AF10071E02418900B70E034FCC3648094804022
:103B010014A3E02418F0900B70E034FCF0900B75D6
:103B1100E004F080D9900B71E0249C900B70E034AC
:103B2100FFC3648094804014A3E0249CF0900B7048
:103B3100E034FFF0900B76E004F080D9900B71E057
:103B410024F6900B70E034FFC364809480400FA38F
:103B5100E024F6F0900B70E034FFF00E80DE900B65
:103B610071E024FF900B70E034FFC36480948040C7
:103B71000FA3E024FFF0900B70E034FFF00D80DE26
:103B8100EF7002810C2430FF900B72E0FBA3E0FA8E
:103B9100A3E0F9EF129E77900B75E02430FF900BB4
:103BA10072E0FBA3E0FAA3E02401F9E43AFAEF1290
:103BB1009E77900B76E02430FF900B72E0FBA3E040
:103BC100FAA3E02402F9E43AFAEF129E77EE2430E8
:103BD100FF900B72E0FBA3E0FAA3E02403F9E43ABF
:103BE100FAEF129E77ED2430FF900B72E0FBA3E019
:103BF100FAA3E02404F9E43AFAEF129E77900B72EB
:103C0100E0FBA3E0FAA3E02405A13E900B75E06080
:103C11006B2430FF900B72E0FBA3E0FAA3E0F9EF15
:103C2100129E77900B76E02430FF900B72E0FBA39D
:103C3100E0FAA3E02401F9E43AFAEF129E77EE24C8
:103C410030FF900B72E0FBA3E0FAA3E02402F9E459
:103C51003AFAEF129E77ED2430FF900B72E0FBA34E
:103C6100E0FAA3E02403F9E43AFAEF129E77900B0D
:103C710072E0FBA3E0FAA3E02404A13E900B76E0FE
:103C810060502430FF900B72E0FBA3E0FAA3E0F94F
:103C9100EF129E77EE2430FF900B72E0FBA3E0FA67
:103CA100A3E02401F9E43AFAEF129E77ED2430FF04
:103CB100900B72E0FBA3E0FAA3E02402F9E43AFAE4
:103CC100EF129E77900B72E0FBA3E0FAA3E02403CE
:103CD100806BEE60382430FF900B72E0FBA3E0FABA
:103CE100A3E0F9EF129E77ED2430FF900B72E0FB19
:103CF100A3E0FAA3E02401F9E43AFAEF129E7790E7
:103D01000B72E0FBA3E0FAA3E024028030ED601126
:103D11002430FF900B72E0FBA3E0FAA3E0F9EF80FF
:103D21000D900B72E0FBA3E0FAA3E0F97430129E50
:103D310077900B72E0FBA3E0FAA3E02401F9E43AE7
:103D4100FAE4129E772290086FEBF0A3EAF0A3E960
:103D5100F0AB05900874E0FA75F010A42421FEE49C
:103D610035F0900878F0A3CEF0A3E4F0A37429F025
:103D7100E4A3F0A3F075088F7509917830F6087601
:103D8100550876C2AF03EFC4333354C0FF08F69031
:103D91000873E0FE1313543F4FF6EEC4333354C09F
:103DA100FF08F6EA1313543F4FF6A3E0C43333542C
:103DB100C0FF08F690086FE0FBA3E0FAA3E024251A
:103DC100F9E43AFA129E3CFE1313543F4FF6EEC447
:103DD100333354C0FF08F690086FE0FBA3E0FAA369
:103DE100E02426F9E43AFA129E3CFE1313543F4FA5
:103DF100F6EEC4333354C008F67D3F7F0D12991699
:103E0100E4F50EF50F7F8F129A75900878A3E0FD07
:103E11007F1B129916900878E05403FD7F1A1299BE
:103E2100169008A0741DF0A3E4F0A37400F0A3742D
:103E310030F0A37408F07B007A0079097D01128FBC
:103E4100927F807E00129831E4F50EF50F7F8F127C
:103E51009A757F5F7E80129831E50F30E3559008A7
:103E61007AA3E0FD7F1B12991690087AE05403FDB6
:103E71007F1A1299167F527E001298317F1C129779
:103E810044EF540FFFC3940340027F03900875E091
:103E9100FBA3E0FAA3E0F9128C627F8F129A75906E
:103EA1000875E0FBA3E0FAA3E0F9129E3C4480FF11
:103EB100029E77E50E30E77590087D7412F0E50EED
:103EC10030E76A90087DE0FF6412706190087CE041
:103ED100FDFBEF2BFBE433FA900874E0FC75F00274
:103EE100A4FFD3EB9FE5F06480F8EA648098400971
:103EF100EC25E0C39D90087DF090087DE0FF9008DF
:103F010075E0FBA3E0FAA3E0F9128C6290087DE072
:103F1100FFFD900876E48DF0129F2690087CE02F3B
:103F2100F0530E7F7F5E7E8012983180917F5F7E9D
:103F310000129831E50F541F600F7F1C129744EF58
:103F4100541F90087DF07F0822E4F50EF50F7F1CC9
:103F5100129744EF541FFF90087DF090087CE0FD1C
:103F61002FFBE433FA900874E0FC75F002A4FFD350
:103F7100EB9FE5F06480F8EA6480984009EC25E065
:103F8100C39D90087DF090087DE0FF900875E0FBEF
:103F9100A3E0FAA3E0F9128C6290087DE0FF90089B
:103FA1007CE02FF0900874E075F002A4FF90087C8B
:103FB100E0B50707E4B5F003FF80027F082290080F
:103FC100C7EBF0A3EAF0A3E9F0E4FF9008CDE0FE2F
:103FD100EFC39E50299008C7E0FBA3E0FAA3E02FAE
:103FE100F9E43AFA129E3CFE9008CAE0FBA3E0FA1B
:103FF100A3E02FF9E43AFAEE129E770F80CD2290DA
:104001000898EBF0A3EAF0A3E9F0E49008A5F053D7
:104011000F7F7F8F129A757F9D129A757D407F1A4F
:104021001299167D3F7F0D1299167F807E0012989E
:10403100317F8F129A75E4F50EF50F7F1BFE1298F2
:1040410031E50F54176002212DE50F20E302415B9A
:104051007B017A0B790E7F01128C62900B0EE0547A
:10406100F81313543FFF7E0090089CEEF0A3EFF08D
:10407100D39420EE9400400990089CE4F0A37420AE
:10408100F090089CA3E0FF900898E0FBA3E0FAA35E
:10409100E02424F9E43AFAEF129E7790089DE02497
:1040A10004F090089CE03400F0E0FEA3E07803C344
:1040B10033CE33CED8F9F0EE90089CF0E0FCA3E0CB
:1040C100FDEC5403444090089FF0EDA3F090089C50
:1040D100E0FEA3E07803CEC313CE13D8F9F0EE903F
:1040E100089CF07B017A08799F9008B77402F07FF1
:1040F1001A128DAEE4F50EF50F7B019008A204F0C3
:10410100A3740BF0A3740FF090089DE024FF80517D
:10411100C390089DE0941290089CE09400404C7F6D
:10412100067E80129831E50F540660089008A57448
:10413100FFF0415B7F1C12974490089BEFF0530EF8
:104141007F9008A2E0FBA3E0FAA3E0F97F12128CB2
:10415100629008A3E475F012129F2690089DE02456
:10416100EEF090089CE034FFF080A57F407E0012C5
:104171009831E50F5415700790089E04F08005E40E
:1041810090089EF07F9F129A757F1C129744EF54FE
:104191001F90089BF0601FE0FFFDC390089DE09D0C
:1041A100F090089CE09400F09008A2E0FBA3E0FAF4
:1041B100A3E0F9128C627D377F0D1299167F807E04
:1041C100001298317F8F129A757D207F1B129916EC
:1041D100E4F50EF50F7F5FFE1298317F1C129744B4
:1041E100EF541FFF60747B017A0B7930128C62905F
:1041F1000898E0FBA3E0FAA3E02424F9E43AFA12D8
:104201009E3CFD9008AA7401F0A3740BF0A3740EF8
:10421100F0A37401F0A3740BF0A37410F0A3740164
:10422100F0A3740BF0A37430F0900898A3E0FAA304
:10423100E0F91237067F0F129744900898E0FBA32C
:10424100E0FAA3E02427F9E43AFAEF129E77900806
:104251009EE060069008A57401F0E4FD7F1A1299B2
:10426100169008A5E0FF2290086BEBF0A3EAF0A3FB
:10427100E9F0A3EDF0E4900874F0900887740AF077
:10428100A37432F0E4FD7F1A1299167D507F1B1240
:104291009916128A04C292D293129CDC90086FE0A4
:1042A100FFA3E0FBA3E0FAA3E0F9A3E0900890F0FC
:1042B100126E81124A1D900885EFF0706C7B01909F
:1042C100089004F0A37408F0A3747DF0A37408F0BF
:1042D100125C8B90086BE0FBA3E0FAA3E02424F9C5
:1042E100E43AFA7408129E7790086BE0FBA3E0FAB7
:1042F100A3E02404F9E43AFA9008CAEBF0A3EAF047
:10430100A3E9F090086BA3E0FAA3E02424F9E43ACE
:10431100FA129E3C9008CDF07B017A087975123F24
:10432100BF9008747401F0819F900885E0B4FD0787
:10433100E4900874F0819F90088974FFF0A3749C45
:10434100F0A374E6F09008867402F090086EE070B5
:1043510002819F900887E0FF900886E0C39F40029A
:10436100819F900888E0FF14F0EF7002819F128A0C
:1043710004C292D293900889A3E0FAA3E0F912A1B2
:1043810058124A1D900885EFF060112403700281D4
:1043910041240260028157900889818C90089074B1
:1043A10001F0A37408F0A3747DF0A37408F07B01FD
:1043B100125C8B900874E075F028A4FFAEF09008B1
:1043C1006BE0FBA3E0FAA3E02FF9EA3EFAE924242B
:1043D100F9E43AFA7408129E7790086BE0FBA3E0C7
:1043E100FAA3E02FF9EA3EFAE92404F9E43AFA9053
:1043F10008CAEBF0A3EAF0A3E9F090086BA3E0FA96
:10440100A3E02FF9EA3EFAE92424F9E43AFA129EEC
:104411003C9008CDF07B017A087975123FBF900876
:1044210074E004F090086EE014F0900886E014F057
:1044310090088974FFF0A3749CF0A374E1F0614CBF
:1044410090088974FFF0A3749CF0A374E1F09008C4
:1044510086E014F0614C900889E0FBA3E0FAA3E048
:10446100F9EB8A8389827BFF7A9C79D7F4700A748D
:10447100D765827004749C6583900889600D74FF10
:10448100F0A3749CF0A374D7F0614C74FFF0A37493
:104491009CF0A374E6F0900886E004F0614C90086B
:1044A10074E07003129C2D900874E0FF227B017A66
:1044B1000B7906900894EBF0A3EAF0A3E9F024024B
:1044C100F9E43AFA129E3C9008A0F0900B0B7401AB
:1044D100F078067C0BFD900894E0FBA3E0FAA3E0E2
:1044E100F97E007F05129DF49008A0E0D39403406B
:1044F10002E4F0900B07E07005900B0904F09008BE
:1045010094E0FBA3E0FAA3E0F9129E3C7002C145DE
:1045110024FA7002A1FC24FE7002A1C11460672478
:10452100FD602924FD6002C1E2E4900897F0A374C4
:10453100C0F0A374F2F0A3744DF0A37401F0A3745E
:1045410004F0A37402F0A37407F0C16BE490089720
:10455100F0A374C0F0A374C2F0900B0AE0700DA335
:10456100F090089A74FAF0E4A3F0800A90089A7423
:104571009AF0A37402F090089C7406F0A37404F0FE
:10458100A37427F0C16BE4900897F0A374C0F0A363
:104591007492F0900B0AE0700EA3F090089A7438B0
:1045A100F0A37401F0800A90089A7441F0A3740397
:1045B100F090089C7405F0A314F0A37437F0C16B5C
:1045C100E4900897F0A374C0F0A37482F0900B0AF2
:1045D100E0700EA3F090089A7477F0A37401F08054
:1045E1000A90089A74E8F0A37403F090089C74068A
:1045F100F0A37404F0A3743BF0806FE4900897F08B
:10460100A374C0F0A37462F0900B0AE0B4010FE44C
:10461100A3F090089A74F4F0A37401F0800A900852
:104621009A7435F0A37405F090089C7407F0A30404
:10463100F0900B07E090089E700574BFF0802B741A
:104641003FF08026E4900897F0A374C2F0A37402AF
:10465100F0A374D0F0A37407F0A3741BF0A3740F3C
:10466100F0A374FFF0E4900B0BF0900B07E025E052
:1046710025E0FF900897E054F34FF054FCFF900BB6
:104681000AE04F900897F0A3E054FCFF9008A0E0E7
:104691004F900898F0900B09E07F0060027F01EFD6
:1046A10025E0FF900899E054FD4FF07B017A0879ED
:1046B100979008B77404F07F01128DAE7F051297B1
:1046C10044EF54F0FF90089BE04FFD7F05129916CF
:1046D1007B017A08799C9008B77403F07F07128DEB
:1046E100AE22124800900869EFF06002E1B412694D
:1046F10026900822E07002A3E0700890086974090E
:10470100F0E1B4128B75900869EFF06002E1B490AA
:104711000A0AE024FE602224FA605214606424082C
:104721006002E1B4900858E0FBA3E0FAA3E0F9903D
:104731000A0BE0FD12746D8042900A0BE06010904C
:104741000858E0FBA3E0FAA3E0F9127AD9801C90A3
:10475100086D7401F0A3740AF0A3740CF09008586A
:10476100E0FBA3E0FAA3E0F9126B6C800E9008580D
:10477100E0FBA3E0FAA3E0F9127B8A900869EFF06D
:10478100803190086D7401F0A3740AF0A37410F0E5
:10479100900858E0FBA3E0FAA3E0F91270F5900845
:1047A10069EFF0900A10E090095AF0900A11E09038
:1047B100095BF0129BE19009577446F0A37405F070
:1047C100900869E0900959F0900A5EE0FBA3E0FAD5
:1047D100A3E02401F9E43AFA129E3C900A5DF0A3A9
:1047E1007401F0A37409F0A37457F00298BC7F051B
:1047F100129744900AD2129740900AD3EFF0229078
:10480100087E7480F0E4900880F0A3F0900824E022
:10481100FCA3E0FD24F0FBEC34FFFAD3EB94E8EACF
:104821009403401BED2410FFE43CFEEF7806CEC359
:1048310013CE13D8F9FF7C007D30129E8980167C3F
:10484100007D30AF03AE02129E89EF7806CEC3130E
:10485100CE13D8F9FF90084BEEF0A3EFF0125F6191
:10486100E4FF128645129BA9AA06AB07900846E011
:10487100FEA3E0FFD394E8EE9403401BEF2420FF56
:10488100E43EFEEF7806CEC313CE13D8F9FF7C00C9
:104891007D30129E89801A900846E0FEA3E0FF7CDD
:1048A100007D30129E89EF7806CEC313CE13D8F95E
:1048B100FFD3EF9BEE9A4045129BA9D3EF94E8EE0C
:1048C1009403401A129BA9EF2418FFE43EFE7C00DA
:1048D1007D30129E9B7C007D41129E89800F129B30
:1048E100A97C007D41129E897D30129E9BC3900858
:1048F10047E09FFF900846E09EFE1287DF90000F81
:10490100E0700C90085CE07003127A277F0A229015
:104911000849A3E090087DF0E490087CF090000F36
:10492100E0FF900849E475F001129F26FCC3E5F011
:104931009FEC94004007E4900849F0A3F0900849E7
:10494100E0FEA3E07802C333CE33CED8F92410F5CC
:104951008274003EF583E0FCA3E0FDA3E0FEA3E04A
:10496100FF90088312A1067F16121D9F900849E04F
:10497100FEA3E024E4F58274003EF583E0D3648075
:104981009458404F900855E0FEA3E0FF90088774CB
:1049910001F0A37408F0A3747EF07B017A08797F9B
:1049A100125800900849E0FEA3E024E4F582740067
:1049B1003EF583E0FF90087EE0FED3EF6480F8EEE1
:1049C100648098400E90087CE004F0E0C394355078
:1049D10002211E900849E0FEA3E024E4F582740060
:1049E1003EF583E0FF90087EE0FED3EF6480F8EEB1
:1049F1006480985010129A0AE490084EF07F0112D8
:104A010086457F002290084E7401F0E4FF1286452E
:104A110090085CE07003127A277F0A22D292D29327
:104A21007B017A0879757D089008A3EBF0A3EAF081
:104A3100A3E9F0A3EDF0E4A3F09008A6E075F00877
:104A4100A4FF9008A8E5F0F0A3EFF0A3E4F0A374AD
:104A510010F0E4A3F0A37480F078AE7C087D017BB4
:104A6100FF7AB1798A7E007F02129DF49008A3E05B
:104A7100FBA3E0FAA3E0F9E4129E777FE87E0361ED
:104A8100139008A8E07002A3E07002611820950558
:104A9100E59130E7F8E59120E77D3081229008A388
:104AA100E0FBA3E0FAA3E0F99008ACE0FFE92FF9FD
:104AB100E43AFA129E3CFF9008ADE04F129E777FD8
:104AC1001E7E001297DB9008A9E024FFF09008A851
:104AD100E034FFF09008ADE0FFC313F07023748061
:104AE100F09008ACE004F09008A3E0FBA3E0FAA387
:104AF100E0F99008ACE0FFE92FF9E43AFAE4129EFC
:104B010077309505E59130E7F8E59120E7097F1EBB
:104B11007E001297DB4182E49008ACF0A37480F030
:104B21009008AAE4F0A37410F09008A8E07002A322
:104B3100E0600261BA9008AAE07002A3E0607A2006
:104B41009505E59130E7F8E59120E76D30811F90FB
:104B510008ACE024AEF582E43408F583C083C0825A
:104B6100E0FF9008ADE0FEEF4ED082D083F07F1ED3
:104B71007E001297DB9008ABE024FFF09008AAE0DA
:104B810034FFF09008ADE0C313F070157480F0901D
:104B910008ACE004F0E024AEF582E43408F583E4E7
:104BA100F07F1E7E001297DB309505E59130E7F826
:104BB1007F1E7E001297DB61361294C49008A8E034
:104BC100FCA3E0FD4C7008A3E07002A3E060179025
:104BD10008A6E075F008A4B5050AECB5F006A374C3
:104BE100FDF0802D80259008A3E0FBA3E0FAA3E06F
:104BF100F9A3E0FD7C001281C3EFF4FFEEF4FE9017
:104C010008AEE06E7003A3E06F60069008A774FF22
:104C1100F09008A7E0FF22900A5D7440F0A37401B0
:104C2100F0A37409F0A37457F09009577444F0A3EA
:104C31007440F0EF6401705D7F01129557124800D6
:104C4100E4900002F0900822F0A3F0EF703F7B01A6
:104C510090086D04F0A37408F0A37426F0E4A3F0A7
:104C6100900857E0900871F0A374FFF0A37499F0D5
:104C7100A374BBF0900119E0900875F07A01791ADC
:104C81007D2D12552E900822EEF0A3EFF0E4900155
:104C910019F0129BE1900002E0FFD3900823E09FFE
:104CA100900822E094005002A1BE900002E0FD7540
:104CB100F028A4243EF582E5F03401F583E0FE24DA
:104CC1000A900958F0EE240290095EF075F028ED83
:104CD100A4241CF582E5F03401F583E090095FF02E
:104CE100900002E075F028A4241DF582E5F034015E
:104CF100F583E0900960F0EF75F028A4241EF974A3
:104D01000135F0FA7B01C0039008CAEBF0A37409E6
:104D1100F0A37461F0900002E075F028A4243EF540
:104D210082E5F03401F583E09008CDF0D003123F25
:104D3100BF900002E075F028A42441F582E5F0342B
:104D410001F583E090095AF0900849E0FEA3E0786C
:104D510002C333CE33CED8F9FBAA062410F58274F0
:104D6100003AF583A3A3A3E0FF90095BEFF0741071
:104D71002BF58274003AF583E0FCA3E0FDA3E0FE8D
:104D8100A3E0FF780812A0E090095CEFF0900849D9
:104D9100E0FEA3E07802C333CE33CED8F92410F578
:104DA1008274003EF583E0FCA3E0FDA3E0FEA3E0F6
:104DB100FF781012A0E090095DEFF0800B90095888
:104DC1007405F0E490095BF0900822E0FEA3E0FF97
:104DD1004E600A900002E0FEC3EF9E8001E490095C
:104DE10059F0900002E004F022FDF0900894E0FFF9
:104DF1003395E0FEEF25E0FFEE33FE746D2FF9747D
:104E01000A3EFA7B019008A8EBF0A3EAF0A3E9F0CF
:104E11009008A8E0FBA3E0FAA3E0F9E4129E7790E2
:104E210008A8E0FBA3E0FAA3E02402F9E43AFAE4DB
:104E3100129E779008A8E0FBA3E0FAA3E02401F911
:104E4100E43AFA7408129E779008A8E0FBA3E0FA0E
:104E5100A3E02403F9E43AFA7408129E77ED90086E
:104E6100A830E70FE0FBA3E0FAA3E0F9129E3C446F
:104E710080800DE0FBA3E0FAA3E0F9129E3C4440E0
:104E8100129E77ED9008A830E60FE0FBA3E0FAA3AD
:104E9100E0F9129E3C4420800DE0FBA3E0FAA3E080
:104EA100F9129E3C4410129E77ED9008A830E50F50
:104EB100E0FBA3E0FAA3E0F9129E3C4408800DE078
:104EC100FBA3E0FAA3E0F9129E3C4404129E77EDA5
:104ED1009008A830E40FE0FBA3E0FAA3E0F9129EEA
:104EE1003C4402800DE0FBA3E0FAA3E0F9129E3CF2
:104EF1004401129E77ED9008A830E314E0FBA3E093
:104F0100FAA3E02402F9E43AFA129E3C44808012AA
:104F1100E0FBA3E0FAA3E02402F9E43AFA129E3C92
:104F21004440129E77ED9008A830E214E0FBA3E024
:104F3100FAA3E02402F9E43AFA129E3C44208012DA
:104F4100E0FBA3E0FAA3E02402F9E43AFA129E3C62
:104F51004410129E77ED9008A830E114E0FBA3E025
:104F6100FAA3E02402F9E43AFA129E3C44088012C2
:104F7100E0FBA3E0FAA3E02402F9E43AFA129E3C32
:104F81004404129E77ED9008A830E014E0FBA3E002
:104F9100FAA3E02402F9E43AFA129E3C4402801298
:104FA100E0FBA3E0FAA3E02402F9E43AFA129E3C02
:104FB1004401129E777F0222900A0AE0600CA3E06E
:104FC10090085CF09001197401F0900957745EF03B
:104FD100A37403F0900A5E7401F0A37409F0A37442
:104FE10057F0900A5D7440F090085CE0900959F028
:104FF1001298BC90085CE07003127A27222222905A
:105001000894EBF0A3EAF0A3E9F0A3EDF0A3741286
:10501100F07F8F129A757F96129A7575088F7509B0
:1050210090900897E0FD2403FFE433FEEF7804CE6F
:10503100A2E713CE13D8F87830F6ED2403540FC449
:1050410054F0440B08F6900897E033333354F8FFDB
:10505100F0900B08E025E0540E44A008F608761203
:10506100900897E0FEC4540F08F6EEC454F008F619
:105071007E05EFC39408403A74302EF8C000E6FD77
:10508100900894E0FBA3E0FAA3E0F9129E3CFCC473
:10509100540F4DD000F60EECC454F0FD74302EF8D0
:1050A100A60574F82FFF900895E475F001129F266C
:1050B10080C074302EF8E6F6900897E0FF131313C2
:1050C100541FF0E02406F0900899E4F0A37400F076
:1050D100A37430F0900897E0D3941A5002219153B1
:1050E1000EBF9008A0741DF0900899E0F9A3E0FAB2
:1050F100A3E09008A1C9F0A3EAF0A3E9F0A3741A10
:10510100F07B007A0079097D01128F92900897E077
:1051110024E6F090089AE475F01A804A900898E025
:10512100FF900897E0D39F40427D0F7C007F007E77
:10513100401291BA530EBF900899E0FBA3E0FAA385
:10514100E0F9900898E09008B7F07F1F128DAE90BB
:105151000897E0FFA3E0FEC3EF9E900897F0EEFFF3
:1051610090089AE48FF0129F2680B17D0F7C007F1A
:10517100007E401291BA900899E0FBA3E0FAA3E007
:10518100F9900897E09008B7F07F1F128DAE802E3E
:105191009008A0741DF0900899E0F9A3E0FAA3E04B
:1051A1009008A1C9F0A3EAF0A3E9F0900897E09074
:1051B10008A4F07B007A0079097D01128F927D0F9E
:1051C1007C007F807E001291BA7F96029A75E490EE
:1051D1000869F0900A0AE0640170677F021295572E
:1051E10012480090086AEFF0E4900000F0128E0679
:1051F10090086AE06009E4900822F0A3F080329000
:105201000A0BE090086FF0A37401F0A3740AF0A3F5
:10521100740CF0900A14E0900873F07B017A017924
:105221001A7D2D124268EF3395E0900822F0A3EF2A
:10523100F0129BE19008587401F0A37401F0A3747B
:105241001AF0E4900869F0900869E0FFC3940F50E8
:105251001474572FF582E43409F583E4F09008695A
:10526100E004F080E29009577440F0A37410F0E478
:1052710090095AF0900000E0FB75F028A4243EF557
:1052810082E5F03401F583E0FA90095BF09008497A
:10529100E0FEA3E07802C333CE33CED8F92410F573
:1052A1008274003EF583E0FCA3E0FDA3A3E0FF9040
:1052B1000964EFF0900849E0FEA3E07802C333CE21
:1052C10033CED8F92410F58274003EF583E0FCA3B7
:1052D100E0FDA3E0FEA3E0FF780812A0E0900965DD
:1052E100EFF0900849E0FEA3E07802C333CE33CE5D
:1052F100D8F92410F58274003EF583E0FCA3E0FDAB
:10530100A3E0FEA3E0FF781012A0E0E4900966EFAD
:10531100F0EA603AEB75F028A4241EF9740135F027
:10532100FA7B01C0039008CAEBF0A37409F0A374DF
:105331005CF0900000E075F028A4243EF582E5F0D1
:105341003401F583E09008CDF0D003123FBF9008FF
:1053510022E0FEA3E0FF4E600E900000E0FEC3EFEE
:105361009E900959F080099009587405F0E4A3F062
:10537100900000E004F0900A5D7410F0A37401F055
:10538100A37409F0A37457F00298BC90086AEBF07B
:10539100A3EAF0A3E9F0A3EDF0900875740DF0E431
:1053A100900874F0FD7F1A1299167D187F1B1299CF
:1053B10016900871E0FF14F0EF7002A11F900874BD
:1053C100E06002A11F128A04C292D293D2937F019C
:1053D1007E001287DF127971900872EFF03395E049
:1053E100FEEF25E0FFEE33FE746D2FF9740A3EFAED
:1053F1007B01900875E0FD124E06900872E02FF0D7
:10540100900875E0A3F0E4900873F090086AE0FB5F
:10541100A3E0FAA3E0F9900873E0FFFD3395E0FC07
:10542100E92DF9EA3CFA129E3CFEEF3395E0FC745B
:10543100772DF58274083CF583EEF0900872E0FF59
:105441003395E0FEEF25E0FFEE33FE746D2FF97426
:105451000A3EFA7B0174772DF58274083CF583E0EE
:10546100FD124E06900872E02FF0A3E004F0E0C3B5
:1054710064809488409590086DE0FD90087FF090DD
:105481000872124DEF900872E02FF090086DE00461
:10549100F0A3E0FBA3E0FAA3E0F9129E3CFD900823
:1054A10080F0900872124DEF900872E02FF0900892
:1054B1006FE475F001129F267B017A0879767D0BE6
:1054C1007C001281C390087212905C900872E02FE8
:1054D100F07B017A0A796DE0FD3395E0FC1298E7E3
:1054E100D293D292D2937B017A0879817D01124ABB
:1054F10029900874EFF0700E900881E07FFC700134
:10550100FF900874EFF0128A04C292D293D2937F73
:105511000F7E001287DF1296141294C461B29008B4
:1055210074E06003129C2D900874E0FF22900869DA
:10553100EBF0A3EAF0A3E9F0A3EDF0E4900876F034
:10554100A3F090087AF0F50EF50F7F8F129A75E4AB
:1055510090087AF090086CE0FF90087AE0C39F50C1
:105561004D900869E0FBA3E0FAA3E0F990087AE026
:10557100FF75F028A4F582E92582F9EA35F0FAE40D
:10558100F5F0129F7DEF75F028A4FF900869E0FB0C
:10559100A3E0FAA3E02FF9EA35F0FAE92424F9E4CB
:1055A1003AFAE4129E7790087AE004F080A6E4F5D6
:1055B1000EF50F900875E0601190086DE0FBA3E017
:1055C100FAA3E0F9A3E0FD1250007F2C7E01129CAA
:1055D10066E4F50EF50F900871E0FF1289879008D7
:1055E1007B7401F0A37499F0E47F01FEFDFC900847
:1055F10071E0F9F812A0F3900878EEF0A3EFF090C3
:10560100086CE0FD900876E0FEA3E0FFC39DEE94F8
:1056110000505E900879E024FFF0900878E034FFB4
:10562100F07C007D28129E89900869E0FBA3E0FAD6
:10563100A3E02FF9EA3EFA90087CE0FD122CB0BFFE
:10564100010E900877E004F07006900876E004F00F
:10565100900872A3E0FAA3E0F912A15890087BEF39
:10566100F0900878E07002A3E0600690087BE0709B
:105671008E7F807E001298317F96129A757F8F12ED
:105681009A75E4F50EF50F900876E07002A3E070CC
:1056910021900B0DE024FFF0900B0CE034FFF0E0C3
:1056A1007002A3E07015FF128645129C2D1244AEC4
:1056B1008000900B0CE4F0A3740AF0900876E0FEF1
:1056C100A3E0FF2290086AEBF0A3EAF0A3E9F0E47B
:1056D100900872F090086AE0FBA3E0FAA3E02425A9
:1056E100F9E43AFA9008907401F0A37408F0A374F5
:1056F10073F01275EA900871EFF06003E0FF227514
:10570100088F900872E0FF7003750990EFB40103F0
:10571100750991E47830F60876570876C490086DDB
:10572100E0FBA3E0FAA3E0F9129E3CFF900873E0CE
:105731006F08F6E92401F9E43AFA129E3CFF900859
:1057410074E06F08F690086AE0FBA3E0FAA3E02496
:1057510025F9E43AFA129E3CFF131313541FFE90ED
:105761000870E0C43354E04E08F690086AE0FBA3E9
:10577100E0FAA3E02426F9E43AFA129E3CFE131360
:1057810013541FFDEFC43354E04D08F6EEC43354F7
:10579100E008F67D367F0D1299167F8F129A75E417
:1057A100F50EF50F9008A0741DF0A3E4F0A37400AA
:1057B100F0A37430F0A37408F07B007A0079097DBE
:1057C10001128F9290086A1282EC900871EFF07DBD
:1057D1003F7F0D129916900871E0FF600122900839
:1057E1006EE475F002129F26900872E004F0E0C3A7
:1057F10094025002C1D57F0022E4900B43F0229025
:105801000884EBF0A3EAF0A3E9F0EEC313FEEF1373
:10581100FF90088EEEF0A3EFF04E700790088EF027
:10582100A304F0E4FF12974490088AEFF07D02E4AC
:10583100FF1299167F0912974490088DEFF07DFFB2
:105841007F0912991690088AE020E1077F0A7E00FD
:105851001287DFE4900890F090088E74FFF5F01243
:105861009F3C45F060481299E490088BEFF0E0FF0F
:10587100C4540FFEEF540F2EFF900891F090089042
:10588100E0FD3395E0FCD3EF9DEC6480F8748098E3
:1058910040C6A3E0900890F090088BE0FF90088448
:1058A100E0FBA3E0FAA3E0F9EF129E7780AA90084B
:1058B10090E0FF701E900887E0FBA3E0FAA3E0F9F7
:1058C1007480129E77900884E0FBA3E0FAA3E0F9CC
:1058D100E4216DEF7803A2E713D8FBFF900890E075
:1058E1002FF07F0A12974490088CEFF07F051297F2
:1058F1004490088CE0FE30E211900890E024B5F06D
:10590100EE30E023E02405F0801D900890E024B9FA
:10591100F0EE30E104E024F6F090088CE030E0078E
:10592100900890E02408F0EF30E71C900890E0FF29
:1059310090088CE0C41313540375F003A4FEC3EF65
:105941009E900890F0801490088CE0C413135403C7
:1059510075F003A4FF900890E02FF0900890E0FF0D
:10596100900887E0FBA3E0FAA3E0F9EF129E77909D
:10597100088DE0FD7F0912991690088A12991290FC
:10598100088AE030E0077F067E001287DF22900B55
:1059910038E024DF7002417314700241912421B474
:1059A1000500400241AB9059B125E05002058373D7
:1059B10021BB21CE21F34122413C900B3374FFF0F6
:1059C100A374A9F0A37416F090A9168065900B3307
:1059D10074FFF0A374A9F0A37428F090A92BE493A9
:1059E100FE90A92AE4937C002400FFEC3E900B403A
:1059F100418B900B39E075F003A42467F582E5F043
:105A0100340BF583E0FBA3E0FAA3E0F9900B33EB51
:105A1100F0A3EAF0A3E9F0129E3CFF900B40E48072
:105A210069900B3374FFF0A374A9F0A37431F09063
:105A3100A931E493FF900B40E4804F900B39E0FFD4
:105A410064817066EF900B33B4811074FFF0A3741E
:105A5100A9F0A37443F090A943800E74FFF0A374DE
:105A6100A9F0A3744AF090A94AE493FF900B40E493
:105A71008018900B3374FFF0A374A9F0A3743AF06B
:105A810090A93AE493FF900B40E4F0A3EFF0801D5E
:105A9100900B3374FFF0A374A9F0A37451F0900B31
:105AA100407403F0A37414F080031217E3900B38D1
:105AB100E0FF64016013EF6402600EEF64036009AC
:105AC100EF64046004EFB40523900B3DE0FFD39035
:105AD1000B41E09F900B40E094004010900B3CE0A4
:105AE100700AE0FE900B40EEF0A3EFF0900B42E065
:105AF10064046018E59620E7FB7596117597409050
:105B01000B427401F0E4900B3EF0A3F02290086D7B
:105B1100EFF0A3ECF0A3EDF0A3EAF0A3EBF0E49037
:105B2100087BF0FE7F2CFDFB7A00793012A33578DB
:105B31003276D490086DE033333354F808F6FDA380
:105B4100E0FAA3E0FBEAFFEF540325E0FFED4FFF8E
:105B5100F6FDEBAE027807CEA2E713CE13D8F854C8
:105B6100014D7833F690086EA3E0FF25E054FE085E
:105B7100F6A3E064827004A3E0646660028105908C
:105B81000870E0FCA3E0FDECC41313135401783456
:105B910046F6EDAE047807CEC313CE13D8F97835A7
:105BA100F6900871E025E0FFE43308A607787C7CD5
:105BB100087D017BFF7AA779857E007F02129DF423
:105BC100900883E4F0A37410F0A3E4F0A37400F050
:105BD100A37436F0A3E4F0A37407F07B017A08798B
:105BE1007CE4FDFC1210479008837401F0A3745605
:105BF100F0A3E4F0A37400F0A37438F0A3E4F0A3DD
:105C010074078054900870E0FCA3E0FDEC131313BB
:105C1100541F783446F6EDAE047803CEC313CE1389
:105C2100D8F97835F6900870E0FEA3E07805C33323
:105C3100CE33CED8F97836F6900870E0FFA3E09025
:105C41000883CFF0A3EFF0A3E4F0A37400F0A374F2
:105C510036F0A3E4F0A37403F0900872E0FBA3E034
:105C6100FAA3E0F9E4FDFC121047900875E0F9A3EE
:105C7100E0FAA3E0900875C9F0A3EAF0A3E9F0A364
:105C8100E4F0A3F0A3F0A3E0FF227A087975E4FD24
:105C910090088CEBF0A3EAF0A3E9F0A3EDF09008F3
:105CA100A27451F0900893E02402F0E0FFD3942015
:105CB1004007EFC41354078001E4FD7F1A129916BF
:105CC100900893E0541F75F008A4FD7F1B129916EC
:105CD100900893E024FEF0128A04C292D293D293E8
:105CE1007F017E001287DF127971900894EFF03303
:105CF10095E0FEEF25E0FFEE33FE746D2FF9740A97
:105D01003EFA7B019008A2E0FD124E06900894E055
:105D11002FF09008A2E0900897F0E4900895F09099
:105D2100088CE0FBA3E0FAA3E0F9900895E0FFFD01
:105D31003395E0FCE92DF9EA3CFA129E3CFEEF3383
:105D410095E0FC74982DF58274083CF583EEF09093
:105D51000894E0FF3395E0FEEF25E0FFEE33FE749B
:105D61006D2FF9740A3EFA7B0174982DF58274083F
:105D71003CF583E0FD124E06900894E02FF0A3E07D
:105D810004F0E0C364809488409590088FE0900807
:105D9100A0124DEA900894E02FF0900893E014903F
:105DA10008A1124DEA900894E02FF07B017A08795E
:105DB100977D0B7C001281C390089412905C90082F
:105DC10094E02FF07B017A0A796DE0FD3395E0FCD8
:105DD1001298E7D293D292D293900890E0FBA3E07D
:105DE100FAA3E0F9A3E0FD124A29900896EFF060CA
:105DF10003129C2D900896E0FF2290087FEBF0A300
:105E0100EAF0A3E9F0E4900885F090087FE0FBA3B5
:105E1100E0FAA3E02425F9E43AFA9008907401F03D
:105E2100A37408F0A37486F01275EAEF6006E4F536
:105E31000EF50F2275088F750990E47830F6087613
:105E4100500876C6900882E0FBA3E0FAA3E0F912BD
:105E51009E3CFF900886E06F08F6E92401F9E43AD8
:105E6100FA129E3CFF900887E06F08F690087FE0E9
:105E7100FBA3E0FAA3E02425F9E43AFA129E3C08D8
:105E8100F690087FE0FBA3E0FAA3E02426F9E43AC8
:105E9100FA129E3C08F67F8F129A75E4F50EF50F03
:105EA1009008A0741DF0A3E4F0A37400F0A3743073
:105EB100F0A37407F07B007A0079097D01128F92BB
:105EC100E4F50EF50F7F5FFE129831E50F20E072C9
:105ED1007F1C129744EF540FFFC3940340027F03CA
:105EE1007B017A087988128C6290087FE0FBA3E03D
:105EF100FAA3E02426F9E43AFA129E3CFF900889BD
:105F0100E06F703690087FA3E0FAA3E02425F9E45E
:105F11003AFA129E3CFF900888E0B5071D7F8F1268
:105F21009A75E4F50EF50F90088375F002129F261D
:105F3100900885E0B401137F0022E4F50EF50F7F90
:105F410002229008857402F0FF22E4F50EF50F900D
:105F51000885E004F0E0C394025002C10B7F0022E7
:105F6100E49008A7F030A102E1FED2A17F0C7E00EF
:105F71001287DFE49008A7F0900AD6E054FCFDE414
:105F8100FF1299169008A67401F09008A6E0FFC3CD
:105F910094195059EF64126013EF6414600EEF64AA
:105FA100156009EF64166004EFB417269008A7E0A6
:105FB100FF04F0EF75F003A424F3F9740A35F0FA45
:105FC1007B019008A6E0FF9008B77403F0128DAE34
:105FD10080139008A6E0FF24D6F582E4340AF58305
:105FE100E0FD1299169008A6E004F0809D7F2C7EBA
:105FF10001129C66127000900AD612991222229008
:10600100087FEDF090087CEBF0A3EAF0A3E9F090B3
:106011000887E4F0A37421F0E92425F9E43AFA9021
:1060210008907401F0A37408F0A37485F01275EA66
:10603100EF6006E4F50EF50F2275088F750991E4FE
:106041007830F60876650876C390087FE0C433336C
:1060510054C0FF08F6A3E0FE1313543F4FF6EEC4FD
:10606100333354C0FF08F6A3E0FBA3E0FAA3E0F941
:10607100129E3CFE900885E06EFE1313543F4FF6CE
:10608100EEC4333354C0FF08F6E92401F9E43AFAC7
:10609100129E3CFE900886E06EFE1313543F4FF6AD
:1060A100AF06EFC4333354C0FF08F690087CE0FB21
:1060B100A3E0FAA3E02425F9E43AFA129E3CFE1388
:1060C10013543F4FF6EEC4333354C0FF08F6900823
:1060D1007CE0FBA3E0FAA3E02426F9E43AFA129E5D
:1060E1003CFE1313543F4FF6EEC4333354C008F64D
:1060F100900887A3E0FD7F1B129916900887E05452
:1061010003FD7F1A1299167D3E7F0D1299167F8F1E
:10611100129A75E4F50EF50F9008A0741DF0A3E432
:10612100F0A37400F0A37430F0A37409F07B007A3B
:106131000079097D01128F9290087CE0FBA3E0FABF
:10614100A3E02425F9E43AFA126D7D900884EFF07A
:106151007D3F7F0D129916900884E0FF22900B83FA
:10616100EBF0A3EAF0A3E9F0A3EDF0E4900B88F0E3
:106171007BFF7AA77912900B87E09008CAF0123062
:1061810000900B83E0FBA3E0FAA3E02401F9E43AD9
:10619100FA129E3C9008CAF0900B83A3E0FAA3E0A8
:1061A100F9129E3C9008CBF07BFF7AA7791D123043
:1061B100007BFF7AA7792E900B86E024029008CA13
:1061C100F0123000900B83E0FBA3E0FAA3E024037C
:1061D100F9E43AFA129E3C9008CAF0900B83A3E0CE
:1061E100FAA3E02402F9E43AFA129E3C9008CBF0BB
:1061F1007BFF7AA779481230007BFF7AA779561284
:106201003000900B86E0FF900B88E0FEC39F50307A
:10621100900B83E0FBA3E0FAA3E02404F9E43AFA4B
:10622100EE7E0029F9EE3AFA129E3C9008CAF07B04
:10623100FF7AA7790A123000900B88E004F080C23F
:106241007BFF7AA77910123000900B83E0FBA3E06B
:10625100FAA3E02424F9E43AFA129E3C9008CAF029
:106261007BFF7AA7795C123000900B83E0FBA3E0FF
:10627100FAA3E02425F9E43AFA129E3C9008CAF008
:10628100900B83A3E0FAA3E02426F9E43AFA129EE4
:106291003C9008CBF07BFF7AA77972023000900A1C
:1062A1000AE0640170547F01129557124800E4908E
:1062B1000001F0900822F0A3F0EF703B7B01900801
:1062C1008204F0A37408F0A37426F0E4A3F090080C
:1062D10057E0900886F0A374FFF0A37499F0A374BB
:1062E100BBF0A37401F07A01791A7D2D123431903B
:1062F1000822EEF0A3EFF0129BE1900A5E7401F028
:10630100A37409F0A37457F0900A5D7440F09009EA
:10631100577432F0900822E0FEA3E0FF4E600A902D
:106321000001E0FEC3EF9E8001E4900959F0900066
:1063310001E0FFD3900823E09F900822E0940050F1
:106341000261CD900001E0FD75F028A4243EF582A4
:10635100E5F03401F583E0FE2406900958F0EE24BF
:106361000290095AF075F028EDA4241CF582E5F09D
:106371003401F583E090095BF0900001E075F028AD
:10638100A4241DF582E5F03401F583E090095CF069
:10639100EF75F028A4241EF9740135F0FA7B01C0D1
:1063A100039008CAEBF0A37409F0A3745DF09000A8
:1063B10001E075F028A4243EF582E5F03401F5836F
:1063C100E09008CDF0D003123FBF800B90095874C4
:1063D10004F0E490095AF0900001E004F022E49006
:1063E1000869F0A3F0900878F0A3F0A3F0A3F012ED
:1063F1004800900869EFF0600281D2126926900886
:1064010022E07002A3E070089008697409F081D25B
:106411007B017A0A790A128B7B900869EFF060029E
:1064210081D2900A0EE0FDC4540FFF90086BE4F096
:10643100A3EFF0E0F8E4F0E890086BF0ED540F758D
:10644100F010A4FFE045F0F0A3E04FF0900A0FE058
:10645100FFC4540FFD90086BE0F0A3E04DF0EF5442
:106461000F7F00FEA3F0A3EFF0900A10E0FDEDFF17
:1064710090086DEEF0A3EFF0A37401F0A3740AF09D
:10648100A37413F0A37401F0A37409F0A3745BF077
:10649100900A11E0900875F0900A12E0900876F0E9
:1064A100E4A3F0FE7F3CFD7B017A09795B12A33501
:1064B10090087F7401F0A37408F0A3746BF0900846
:1064C10058E0FBA3E0FAA3E0F9122800900869EF75
:1064D100F0129BE19009577460F0A37440F09008AA
:1064E10069E0900959F0900877E090095AF07B0132
:1064F1007A097957900A5EEBF0A3EAF0A3E9F02458
:1065010001F9E43AFA129E3C900A5DF00298BCE46B
:1065110090086AF0900A0CE0900869F01248009027
:10652100086AEFF06002C107126926900822E07044
:1065310002A3E0700890086A7409F0C10790086925
:10654100E06002A1D57B0190086B04F0A37409F00F
:10655100A3745BF0900A0BE090086EF090086AE07B
:10656100705E900869E0C3941E50551299BBEF60AC
:106571004F900A0AE0FD90086EE0FF04F090087366
:10658100EFF0A37401F090086BE0F9A3E0FAA3E047
:10659100900875C9F0A3EAF0A3E9F0900858E0FB70
:1065A100A3E0FAA3E0F9123D4790086AEFF09008E2
:1065B10069E004F090086CE475F002129F26809C5B
:1065C100900869E014F090084EE0603A90086A740F
:1065D1000AF08032900A0AE0FDA3E0900873F0907F
:1065E1000869E0900874F0A37401F0A37409F0A3A2
:1065F100745BF0900858E0FBA3E0FAA3E0F9123DC8
:106601004790086AEFF0129BE19009577438F090B7
:10661100086AE0900959F0900869E0FD25E024043A
:10662100900958F090095AEDF0900A5D7440F0A37A
:106631007401F0A37409F0A37457F00298BC1248D6
:106641000090086CEFF06002E12D1269269008229B
:10665100E07002A3E0700890086C7409F0E12D125B
:106661008B7590086CEFF06002E12D900A0AE0FF53
:10667100B401057402F0800AEFB40206900A0A74AC
:1066810001F0E4900869F0A3F0A3F0900A0BE0FD9B
:10669100701090086974C0F0900A0AE0FEC454308A
:1066A100802BEDB401139008697430F0900A0AE070
:1066B100FF25E025E0540C8014900A0BE0FDB402A4
:1066C10012900869740CF0900A0AE0540390086A69
:1066D100F08038EDB403129008697403F0900A0A4F
:1066E100E0FFC4333354C08015900A0BE0B40414A6
:1066F10090086A74C0F0900A0AE0FFC45430900810
:106701006BF08007E4900869F0A3F09008707401C1
:10671100F0A37408F0A37469F0900858E0FBA3E0BB
:10672100FAA3E0F91272C990086CEFF0129BE190A4
:106731000957743CF0A37404F090086CE090095977
:10674100F0900A5EE0FBA3E0FAA3E02401F9E43A49
:10675100FA129E3C900A5DF0A37401F0A37409F053
:10676100A37457F00298BC900869EFF0D3940F40DE
:10677100037489F0900869E02457F582E4340BF53D
:1067810083E090086BF0E0C413540790086AF0901E
:10679100086AE0FFD39400404DC2A2EF14FF7401D8
:1067A1007E00A807088005C333CE33CED8F9FF9009
:1067B100086BE0FDEF5D7BFF600D7AA6797A123000
:1067C100007FC27E01800B7AA6797C1230007FFAAD
:1067D1007E001287DFD2A27F5E7E011287DF9008E2
:1067E1006AE014F080A97BFF7AA6797E900869E0BF
:1067F1009008CAF01230007FC27E010287DF22E4D6
:10680100900869F0128E06124800900869EFF0E4D2
:10681100900822F0A3F0EF600201D190086B04F020
:10682100900882F0A3740AF0A3740BF0900A0AE0B6
:10683100900885F0E4A3F0A374FFF0A37499F0A38A
:1068410074BBF0A37401F0FB7A01791AFD123431A3
:10685100900822EEF0A3EFF0E490086AF0900A0AA3
:10686100E0FF90086AE0FEC39F501A740B2EF58278
:10687100E4340AF583E06005E490086BF090086A5F
:10688100E004F080D8900822E07002A3E07041900B
:10689100086BE0603B9008827401F0A3740AF0A3D6
:1068A100740BF0A3EFF0900857E0900886F0A37402
:1068B100FFF0A37499F0A374BBF0E4A3F07B017A19
:1068C10001791A7D01123431900822EEF0A3EFF024
:1068D100129BE1900822E07002A3E0900858601238
:1068E1007401F0A37401F0A3741AF0E4900869F044
:1068F100800CE4F0A3F0A3F09008697409F090090A
:10690100577434F0A37403F0900869E0900959F0CA
:10691100900A5D7403F0A37401F0A37409F0A374E9
:1069210057F00298BC900858A3E0FAA3E04A70031C
:10693100FEFF22900858E0FBA3E0FAA3E02404F94B
:10694100E43AFA900882EBF0A3EAF0A3E9F09008A8
:1069510058A3E0FAA3E02424F9E43AFA129E3C9009
:106961000885F0E4A3F0A374FFF0A37499F0A37475
:10697100BBF0A37401F0FB7A017942FD123431902E
:106981000822EEF0A3EFF090087D7401F0E4900886
:106991007CF0900858E0FBA3E0FAA3E02424F9E49A
:1069A1003AFA129E3CFF90087CE0FEC39F5028906B
:1069B1000858A3E0FAA3E02404F9E43AFAEE7C00D3
:1069C10029F9EC3AFA129E3C6005E490087DF090BA
:1069D100087CE004F080BB900822E07002A3E07024
:1069E1004E90087DE06048900858E0FBA3E0FAA3D0
:1069F100E02404F9E43AFA900882EBF0A3EAF0A368
:106A0100E9F0A3EFF0900857E0900886F0A374FF37
:106A1100F0A37499F0A374BBF0E4A3F07B017A01B5
:106A210079427D01123431900822EEF0A3EFF0900B
:106A31000822E07002A3E0600E9008587401F0A3F0
:106A41007401F0A37442F02290084DE024FD604BE4
:106A5100147002611E24026002615AE490000AF07F
:106A6100FFFEFDFC90000612A106900A097402F0D7
:106A7100121027EF70026160129CBF90000AE0FEC5
:106A810004F074082EF582E4340AF583EFF09008DF
:106A91004D7403F0E490085CF06160900006E0FC46
:106AA100A3E0FDA3E0FEA3E0FFE4FAF9F8EF24017F
:106AB100FFEA3EFEE93DFDE83CFC90000612A1061E
:106AC100E4FF7E80FDFC900006E0F8A3E0F9A3E07E
:106AD100FAA3E0FBD312A0B9501390000AE0FF948F
:106AE1003F500A900A09E0FEEFC39E400790084D0F
:106AF1007404F022121027EF6065129CBF90000A07
:106B0100E0FE04F074082EF582E4340AF583EFF018
:106B1100E4FFFEFDFC90000612A10680427F40903A
:106B21000957E4F0A3DFFC7F4090084D7402F09018
:106B3100084814F0125F61900A08E075F003A4247C
:106B410086F582E5F034ACF583740193FA7402930F
:106B5100F912A158E4900848F090084D7402F090A1
:106B6100085CE060057F01129BCF2290086AEBF080
:106B7100A3EAF0A3E9F02425F9E43AFA9008907425
:106B810001F0A37408F0A37471F01275EAEF6006C6
:106B9100E4F50EF50F2275088F750991E47830F64A
:106BA1000876800876E008760290086DE0FBA3E0A5
:106BB100FAA3E0F9129E3CFF900871E0FE6F08F61F
:106BC100E92401F9E43AFA129E3CFF900872E0FDD3
:106BD1006F08F690086DE0FBA3E0FAA3E02402F948
:106BE100E43AFA129E3CFFEE6F08F690086DE0FB66
:106BF100A3E0FAA3E02403F9E43AFA129E3CFFED84
:106C01006F08F690086AE0FBA3E0FAA3E02425F9F7
:106C1100E43AFA129E3C08F690086AE0FBA3E0FA17
:106C2100A3E02426F9E43AFA129E3C08F67D367F69
:106C31000D1299167F8F129A75E4F50EF50F9008D3
:106C4100A0741DF0A3E4F0A37400F0A37430F0A3CA
:106C5100740AF07B007A0079097D01128F92900805
:106C61006A1282EC900870EFF07D3F7F0D12991649
:106C7100900870E0FF2290087CEFF07F05129744A6
:106C810090087E12974090087DEFF0543CF030E27E
:106C91001A90087CE02448F0E0D364809485403762
:106CA100E024FBF0A3E04401F0802C90087CE02478
:106CB10042F0E0C3648094884009E024F8F0A3E046
:106CC1004401F090087CE0D3648094765009E0247C
:106CD1000AF0A3E04402F090087CE0FDD3648094C4
:106CE10080403190087EE0547FF0ED75F003129EF4
:106CF1001A90087FF0D3940340037403F090087C4A
:106D0100E0FF90087FE075F003A4FEC3EF9E9008BA
:106D11007CF0803B90087EE04480F090087CE0FFAE
:106D21003395E0FEC374029FFFE49EFE7C007D0369
:106D3100129EF090087FEFF0D3940340037403F0A8
:106D410090087FE075F003A4FF90087CE02FF0909D
:106D5100087DE0FF90087FE0C4333354C0FEEF4E5E
:106D610090087DF0A3E0FD7F0512991690087DE063
:106D7100FD7F0A12991690087CE0FF22900889EBAA
:106D8100F0A3EAF0A3E9F0A37404F0900890E4F012
:106D9100A37429F07F807E00129831E4F50EF50F7F
:106DA1007F8F129A757D147C007F5A7E001291BAF2
:106DB100E50F30E355900890A3E0FD7F1B12991673
:106DC100900890E05403FD7F1A1299167F527E00BD
:106DD1001298317F1C129744EF540F900892F0C320
:106DE100940340037403F0900892E0FF7B017A085A
:106DF100798D128C627F8F129A757D3F7F0D12996A
:106E01001690088DE04480FFF022E50F30E6567FB2
:106E11001C129744EF540F900892F0C39402400360
:106E21007402F0900892E0FF7B017A08798D128C50
:106E3100627F8F129A75900889E0FBA3E0FAA3E0C4
:106E4100F9129E3CFF90088DE06F6012E92401F970
:106E5100E43AFA129E3CFF90088EE0B50717E490E1
:106E6100088CF08010E50F90088C30E405740BF06D
:106E710080037404F0E4F50EF50F90088CE0FF2216
:106E810090088DEBF0A3EAF0A3E9F0AC0712797159
:106E910090089CEFF0E4900891F0EF3395E0FEEF5D
:106EA10025E0FFEE33FE746D2FF9740A3EFA7B0183
:106EB100E4FD124E0690089CE02FF0900890E090BF
:106EC1000892F0FD90089C124DEF90089CE02FF085
:106ED100AF04900893EFF0FD90089C124DEF9008DD
:106EE1009CE02FF0A37403F090089DE0FFC3648041
:106EF100948B505B90088DE0FBA3E475F001129F29
:106F01003CA9F0FA129E3CFEEFFD3395E0FC749132
:106F11002DF58274083CF583EEF090089CE0FF3378
:106F210095E0FEEF25E0FFEE33FE746D2FF9740A54
:106F31003EFA7B0174912DF58274083CF583E0FDE6
:106F4100124E0690089CE02FF0A3E004F080997B9C
:106F5100017A0879917D0B7C001281C3AD07AC06E3
:106F610090089C12906090089CE02FF07B017A0AB7
:106F7100796DE0FD3395E0FC0298E790086974FFB4
:106F8100F0124800900869EFF07029900A12E0FDB4
:106F91009008907401F0A37409F0A3745BF0900A57
:106FA10013E0900893F07B017A0A790A125C9190C0
:106FB1000869EFF0129BE1900957744AF0A37440FD
:106FC100F0900869E0FF3395E0FE7CFF7DFF129EA3
:106FD10089900959EFF0900A13E090095AF07B016A
:106FE1007A097957900A5EEBF0A3EAF0A3E9F0245D
:106FF10001F9E43AFA129E3C900A5DF00298BC90C5
:107001000AF2E0700201F47B017A0879A87D037F1E
:10701100121293EE9008AAE054FEF09008A9E054F1
:107021003FF04440F07B017A0879A89008B77403D7
:10703100F07F12128DAEE49008ACF0A3F09008AD91
:10704100E004F070069008ACE004F07F647E00126A
:107051009C667F0E1297449008ABEFF020E10FC3BE
:107061009008ADE094649008ACE0940040CF7A08B9
:1070710079A81293E89008A9E04408128D9F7FC86F
:107081007E00129C667F10129744EF54079008AE61
:10709100F09008A9E054F7128D9F9008AEE0FFD35D
:1070A10094014005EF9406404AE49008ACF0A3F047
:1070B1009008ADE004F070069008ACE004F0900890
:1070C100A9E0547F128D9F9008A9E04480128D9F02
:1070D1007F0A7E001287DF7F0E1297449008ABEF84
:1070E100F020E10FC39008ADE094039008ACE09468
:1070F1000040BD2290086AEBF0A3EAF0A3E9F02476
:1071010025F9E43AFA9008907401F0A37408F0A309
:107111007470F01275EAEF6006E4F50EF50F227552
:10712100088F750991E47830F60876700876E008E2
:10713100760708F690086DE0FBA3E0FAA3E0F912E8
:107141009E3CFF900870E06F08F6E92401F9E43AEB
:10715100FA129E3CFF900871E06F08F690086AE011
:10716100FBA3E0FAA3E02425F9E43AFA129E3C08D5
:10717100F690086AE0FBA3E0FAA3E02426F9E43ADA
:10718100FA129E3C08F67D367F0D1299167F8F12FA
:107191009A75E4F50EF50F9008A0741DF0A3E4F0C4
:1071A100A37400F0A37430F0A37409F07B007A009B
:1071B10079097D01128F9290086AE0FBA3E0FAA39E
:1071C100E02425F9E43AFAC002C001A3E0F9A3E002
:1071D100FAA3E0900875C9F0A3EAF0A3E9F0D001A1
:1071E100D00212780022900BA3EFF0A37403F0A356
:1071F10074E8F0900A5DE0FFA3E0FBA3E0FAA3E0EE
:107201002401F9E43AFAEF129E77900B43E064010E
:107211007031900B43E0B40117900BA474FFF5F0AB
:10722100129F2645F060097F647E00129C6680E211
:10723100900BA4E07002A3E070097BFF7AA879E8C3
:10724100123000E4900BA3F0A2AF9200C2AFE5961A
:1072510020E7FB75960E759701E59620E7FB75967D
:1072610091E59620E7FBAF97900B43E0FEB4030D49
:10727100E59620E7FB7596117597108046EE7043F1
:10728100900B4304F0EF30E50BE59620E7FB759694
:1072910011759740EF30E20BE59620E7FB759611EB
:1072A100E4F597900A5DE0FD7C00A3E0FBA3E0FA22
:1072B100A3E0F97F211290B8E59620E7FB759611BE
:1072C100759701A20092AF2290086DEBF0A3EAF04E
:1072D100A3E9F075088F750991E47830F6087659BD
:1072E1000876C5A3E0FBA3E0FAA3E0F9129E3C08EF
:1072F100F6E92401F9E43AFA129E3C08F690086D89
:10730100E0FBA3E0FAA3E02425F9E43AFA129E3C5B
:10731100FFC4540FFE900870E0FBA3E0FAA3E02441
:1073210002F9E43AFA129E3C54F04E08F690086DC8
:10733100E0FBA3E0FAA3E02426F9E43AFA129E3C2A
:10734100FEC4540FFDEFC454F04D08F6EEC454F0E2
:1073510008F67D367F0D1299167F8F129A75E4F526
:107361000EF50F9008A0741DF0A3E4F0A37400F0D3
:10737100A37430F0A37408F07B007A0079097D01D1
:10738100128F9290086D1282EC900873EFF07D3F9E
:107391007F0D129916900873E0FF22E490086CF0BB
:1073A100900A09E090086BF012480090086CEFF029
:1073B100E07076126926900822E07002A3E070085E
:1073C10090086C7409F08061128B7590086CEFF075
:1073D100E07056900A10E0900869F0FE900A0BE008
:1073E100FF9008717401F0A3740AF0A37411F0A363
:1073F100EEF0900A0AE0900875F0A37401F0A3740E
:1074010008F0A3746CF0900858E0FBA3E0FAA3E045
:10741100F91278B990086AEFF0900869E06F600995
:1074210090086CE0700374FFF0129BE190095774AF
:1074310036F0A37404F090086CE0900959F09008BC
:107441006AE090095AF0900A5EE0FBA3E0FAA3E03B
:107451002401F9E43AFA129E3C900A5DF0A374010A
:10746100F0A37409F0A37457F00298BC90086AEB7A
:10747100F0A3EAF0A3E9F075088F750991E478307B
:10748100F60876430876E0087603ED600508768015
:107491008004E47834F690086AE0FBA3E0FAA3E004
:1074A1002425F9E43AFA129E3CFF54FEC3137834C2
:1074B10046F6EF5401C43333335480FF90086AE039
:1074C100FBA3E0FAA3E02426F9E43AFA129E3CFE7B
:1074D10054FEC3134F08F6EE5401C43333335480C2
:1074E10008F67D367F0D1299167F8F129A75E4F595
:1074F1000EF50F9008A0741DF0A3E4F0A37400F042
:10750100A37430F0A37407F07B007A0079097D0140
:10751100128F9290086A1282EC90086DEFF07D3F15
:107521007F0D12991690086DE0FF22900B38E070E4
:1075310010A3E0700C900B3CE07006A3E0640260C5
:10754100031217E3900B36E0247F6013146032249A
:10755100027072900B3AE0706CA3E0601580669047
:107561000B32E0B4040A900B3AE07004A3E060022D
:107571008053900B3374FFF0A374B1F0A37488802F
:1075810036900B32E0B40406900B3AE0600280358D
:10759100900B3BE0B4812C900B43E0900B33B40390
:1075A1000C74FFF0A374B1F0A37486800A74FFF029
:1075B100A374B1F0A37488F0900B40E4F0A37402BB
:1075C100F0800580001217E3900B42E0640460181C
:1075D100E59620E7FB759611759740900B42740173
:1075E100F0E4900B3EF0A3F0229008937401F07543
:1075F100088F750990E47830F60876300876C11264
:107601009E3C08F6E92401F9E43AFA129E3C08F698
:10761100E4F50EF50FFD7F1A1299167D207F1B12DE
:1076210099167F8F129A759008A0741DF0A3E4F04B
:10763100A37400F0A37430F0A37405F07B007A000A
:1076410079097D01128F927F807E001298317F8FA0
:10765100129A757F5F7E00129831E50F30E628E5BA
:107661000F541E60089008937401F08024E4F50E15
:10767100F50F900890E0FBA3E0FAA3E0F9129CEB70
:10768100E4900893F0800AE4F50EF50F9008930456
:10769100F0E4FD7F1B129916E4F50EF50F900893A7
:1076A100E0FF22900869E4F0A3F0A3F0900AF2E071
:1076B100B4011090086974FFF0A374A8F0A37416C4
:1076C100F08038900A0AE014601304702090086971
:1076D10074FFF0A374A8F0A3742AF0801E900869C7
:1076E10074FFF0A374A8F0A37448F0800E900869A9
:1076F10074FFF0A374A8F0A3746CF07F3190095962
:10770100E4F0A3DFFC9009577411F0900869E0FBE5
:10771100A3E0FAA3E0F91227DBEF04900958F090F7
:1077210008CA7401F0A37409F0A37459F0900958C0
:10773100E024FE9008CDF0900869E0FBA3E0FAA3F5
:10774100E0F9123FBF900A5E7401F0A37409F0A33F
:107751007457F0900A5D7431F00298BCE4FF1297FF
:1077610044900883EFF07B017A08797F1293EA90C5
:10777100087FE0900882F054CF90087FF07B017A77
:1077810008797F128DA6900883E0440254FEFDE43F
:10779100FF1299167F96129A757F97129A757D013D
:1077A1007F111299167F027E001287DF129968906D
:1077B100087EEFF07D027F111299167F027E001282
:1077C10087DF129968EFFE90087EE0FDEDFF9008DB
:1077D1007CEEF0A3EFF07B017A08797F1293EA90B7
:1077E1000882E090087FF07B017A08797F128DA6EC
:1077F10090088312991290087CE0FEA3E0FF22908A
:107801000872EBF0A3EAF0A3E9F09008787404F0B1
:107811007F807E00129831E4F50EF50F7F8F129A6A
:10782100757D3F7F0D1299167D147C007F527E007D
:107831001291BAE50F30E675900875E0FBA3E0FA06
:10784100A3E0F97F02128C627B017A0879797F02C9
:10785100128C627F8F129A75E50F30E323900875C1
:10786100E0FBA3E0FAA3E0F9129E3C4480129E776C
:10787100900875E0FBA3E0FAA3E0F9129E3C802991
:10788100900872E0FBA3E0FAA3E0F9129E3CFF909E
:107891000879E06F6012E92401F9E43AFA129E3C9A
:1078A100FF90087AE0B50705E4900878F0E4F50E5A
:1078B100F50F900878E0FF2290086DEFF0A3EBF050
:1078C100A3EAF0A3E9F0E4900879F0A3F09008743A
:1078D100E0FF90087AE0C39F4002216BE4A3F0909F
:1078E100087AE0FC90086DE02C900880F0EC75F0CF
:1078F10002A4FF900871E0FBA3E0FAA3E02FF9EAEC
:1079010035F0FA900881EBF0A3EAF0A3E9F09008D2
:1079110075E0FD90086EE0FBA3E0FAA3E0F91260C8
:1079210000900879EFF090087BE004F0E0C3940741
:10793100500C900879E060061299BBEF70A1900895
:107941004EE06006900879740AF0900879E0FF60D3
:1079510011900876E0FBA3E0FAA3E0F9EF129E771D
:10796100800890087AE004F001CE90087AE0FF22C6
:107971007B017A0A796D9008A3EBF0A3EAF0A3E901
:10798100F09008A3E0FBA3E0FAA3E0F97455129E7E
:10799100779008A3E0FBA3E0FAA3E02402F9E43A1C
:1079A100FA7455129E779008A3E0FBA3E0FAA3E0D6
:1079B1002404F9E43AFA7473129E779008A3E0FB69
:1079C100A3E0FAA3E02406F9E43AFA740A129E77D6
:1079D1009008A3E0FBA3E0FAA3E02401F9E43AFA5A
:1079E1007408129E779008A3E0FBA3E0FAA3E024B9
:1079F10003F9E43AFA7408129E779008A3E0FBA316
:107A0100E0FAA3E02405F9E43AFA7408129E7790AB
:107A110008A3E0FBA3E0FAA3E02407F9E43AFA742F
:107A210004129E77FF22E49008A7F020A10241D81A
:107A3100E4FF129744900AD6EFF054FCFDE4FF12E4
:107A410099169008A67401F09008A6E0FFC3941956
:107A51005059EF64126013EF6414600EEF64156007
:107A610009EF64166004EFB417229008A7E0FF0441
:107A7100F0EF75F003A424F3F9740A35F0FA7B01F1
:107A81009008A6E0FF7D031293EE80179008A6E010
:107A9100FF1297449008A6E024D6F582E4340AF553
:107AA10083EFF09008A6E004F0809D9008A874018F
:107AB100F0A374F4F09008A874FFF5F0129F3C4510
:107AC100F060127F0E129744EF30E2097F017E00D1
:107AD1001287DF80E0C2A12290086AEBF0A3EAF0EE
:107AE100A3E9F02425F9E43AFA9008907401F0A38F
:107AF1007408F0A3746EF01275EAEF6006E4F50EF7
:107B0100F50F2275088F750991E47830F6087640F3
:107B11000876E008760190086AE0FBA3E0FAA3E0AA
:107B21002425F9E43AFA129E3C08F690086AE0FB33
:107B3100A3E0FAA3E02426F9E43AFA129E3C08F6FF
:107B41007D367F0D1299167F8F129A75E4F50EF529
:107B51000F9008A0741DF0A3E4F0A37400F0A374C7
:107B610030F0A37406F07B007A0079097D01128F51
:107B71009290086A1282EC90086DEFF07D3F7F0DC4
:107B810012991690086DE0FF2290086AEBF0A3EAC3
:107B9100F0A3E9F02425F9E43AFA9008907401F091
:107BA100A37408F0A3746EF01275EAEF6006E4F5B1
:107BB1000EF50F2275088F750991E47830F6087675
:107BC100400876E008760590086AE0FBA3E0FAA396
:107BD100E02425F9E43AFA129E3C08F690086AE09E
:107BE100FBA3E0FAA3E02426F9E43AFA129E3C084A
:107BF100F67D367F0D1299167F8F129A75E4F50E78
:107C0100F50F9008A0741DF0A3E4F0A37400F0A395
:107C11007430F0A37406F07B007A0079097D0112BB
:107C21008F9290086A1282EC90086DEFF07D3F7F91
:107C31000D12991690086DE0FF22900B8EEBF0A3C8
:107C4100EAF0A3E9F0900B8EE0FBA3E0FAA3E024B5
:107C510002F9E43AFA129E3C9008CAF0900B8EA306
:107C6100E0FAA3E02403F9E43AFA129E3C9008CB2F
:107C7100F07BFF7AA679EB1230007BFF7AA679FFC1
:107C8100123000E4900B91F0A3F0900B8EE0FBA377
:107C9100E0FAA3E02424F9E43AFA129E3CFF900BA7
:107CA10091E0FCA3E0FDC39FEC94005034900B8E57
:107CB100A3E0FAA3E02404F9E43AFAE92DF9EA3C55
:107CC100FA129E3C9008CAF07BFF7AA7790A12301B
:107CD10000900B92E004F070B1900B91E004F08001
:107CE100A97BFF7AA7791002300090085BE0B4010C
:107CF10002E4F0900A0AE06006A3E090084FF090D9
:107D01000A0CE06006A3E0900850F0900A0EE060D3
:107D110006A3E0900851F0900A10E06006A3E090FD
:107D21000852F0900A12E06006A3E0900853F09028
:107D31000A14E06006A3E0900857F07E007F407DC2
:107D4100007B017A09795712A335900957745AF0CB
:107D5100A37440F090084FE090095AF0900850E069
:107D610090095CF0900851E090095EF0900852E0B3
:107D7100900960F0900853E0900962F0900857E094
:107D8100900964F0900A5D7440F0A37401F0A3744B
:107D910009F0A37457F00298BCC0E0C0F0C083C0E2
:107DA10082C0D075D000C000C001C002C003C004B1
:107DB100C005C006C007E59620E7FB759686E596E7
:107DC10020E7FB9008C3E597F0E59620E7FB759661
:107DD10082E59620E7FB9008C4E597F0E59620E759
:107DE100FB759684E59620E7FB9008C5E597F09032
:107DF10008C3E030E103129BF39008C3E030E203D3
:107E01001210079008C4E030E0031224CD9008C49A
:107E1100E030E1031257FA9008C5E030E103127F28
:107E21008B9008C3E030E003129C02D007D006D04B
:107E310005D004D003D002D001D000D0D0D082D060
:107E410083D0F0D0E032E4900869F0A3F0A3F0A36E
:107E5100F0900A0BE090086AF0A3E4F0900A0CE0BD
:107E6100FF90086AE0F0A3E04FF0900A0DE0FAA35A
:107E7100E0FFEFFB900A0AE0FF90086AE0FCA3E054
:107E8100FD9008727401F0A3740AF0A3740FF0A3BB
:107E91007401F0A37409F0A3745BF0A37401F0A35F
:107EA1007408F0A3746CF0125B0E900869EFF01285
:107EB1009BE1900957744EF0A37440F0900869E07B
:107EC100900959F090086CE090095AF07B017A0909
:107ED1007957900A5EEBF0A3EAF0A3E9F02401F9E7
:107EE100E43AFA129E3C900A5DF00298BCE4900BD1
:107EF1008AF0E4900B8BF0A3F0A3F0900B89F09043
:107F01000882E4F0A3F0A3F0A3F0900B8AE09008BC
:107F110086F0A374FFF0A3749CF0A374FAF0A37429
:107F210001F0FB7A01791A7D10123431EFFD900BCB
:107F31008DE02DF0900B8CE03400F0900B8BE0FE87
:107F4100EFD39E4002EFF0900B89E004F0E0C39480
:107F5100FF40AC7BFF7AA6794F900B8AE09008CA6C
:107F6100F0900B8CE0FFA3E09008CBCFF0A3EFF0F3
:107F7100900B8BE09008CDF0123000900B8AE0045A
:107F8100F0E0C3940F5002C1F322E49008C6F0E57B
:107F91009620E7FB75960E759701E59620E7FB7530
:107FA1009694E59620E7FBAF97900B43E0B4030C62
:107FB100E59620E7FB75961475972022EF30E60BC6
:107FC100E59620E7FB75961475978012102F900A9D
:107FD10048E0FD7C00A37F21128F32900A49E0FB2B
:107FE100A3E0FAA3E0F9129E3CFF129000E596206F
:107FF100E7FB759614E4F59722900A5CE0FF22E412
:10800100900B98F0900B98E0FFC3941F40020196EB
:108011007BFF7AA4791A9008CAEFF0123000900B16
:1080210098E0FF64126014EF6414600FEF64156050
:108031000AEF64166005EF6417703C7B017A0B79D7
:10804100997D031293EE7BFF7AA47927900B9BE035
:108051009008CAF01230007BFF7AA47927900B9A1E
:10806100E09008CAF01230007BFF7AA47927900BC8
:1080710099E09008CA8012900B98E0FF1297447B18
:10808100FF7AA4792D9008CAEFF0123000900B9876
:10809100E004F0010522E4FF129744900882129354
:1080A100E290087EE0900881F054CF90087EF07B4A
:1080B100017A08797E128DA6900882E04403FDE4DE
:1080C100FF1299167F96129A757F97129A757D0104
:1080D1007F111299167F027E001287DF129968EFD5
:1080E1003395E090087CF0A3EFF07D027F111299A7
:1080F100167F027E001287DF129968EFFE90087DDD
:10810100E0FDEDFF90087CEEF0A31293E290088170
:10811100E090087EF07B017A08797E128DA69008A6
:108121008212991290087CE0FEA3E0FF2290095789
:10813100741DF0900A0AE0FF64126013EF6414608A
:108141000EEF64156009EF64166004EFB417287B25
:10815100017A0879697D031293EE9008CA7401F0DF
:10816100A37409F0A37459F0A37403F07B017A0896
:108171007969123FBF802E900A0AE0FF129744905E
:108181000869EFF09008CA7401F0A37409F0A374B0
:1081910059F0A37401F0FB7A087969123FBFE490AA
:1081A100095AF0A3F0900957741DF0A37406F090DA
:1081B1000A5DF0A37401F0A37409F0A37457F002EF
:1081C10098BC9008B0EBF0A3EAF0A3E9F0A3ECF0BF
:1081D100A3EDF074FF9008B7F0A3F0E49008B5F0B8
:1081E100A3F09008B3E0FEA3E0FFC39008B6E09FC0
:1081F100EE6480F89008B5E064809850519008B022
:10820100E0FBA3E475F001129F3CA9F0FA129E3C39
:10821100FD9008B7E0FAA3E0FBEAFFEF6D25E0FF70
:10822100E433FE74862FF58274AF3EF583EBFEE4F2
:10823100936EFF7401939008B7CFF0A3EFF090080D
:10824100B6E004F0709C9008B5E004F080949008CA
:10825100B7E0FEA3E0FF2290086A7402F09009578C
:108261007458F0E4900869F0900869E0FFC3941F26
:10827100505AEF64126013EF6414600EEF641560DE
:1082810009EF64166004EFB4171D90086AE07C00E2
:108291002457F9EC3409FA7B017D031293EE90081F
:1082A1006AE02403F0801D900869E0FF1297449072
:1082B100086AE02457F582E43409F583EFF0900869
:1082C1006AE004F0900869E004F0809C90086AE09C
:1082D1002402900958F0900A5D7440F0A37401F0F3
:1082E100A37409F0A37457F00298BCE0FBA3E0FA71
:1082F100A3E02425F9E43AFA900875EBF0A3EAF03B
:10830100A3E9F0A37404F07F807E00129831E4F5B4
:108311000EF50F7F8F129A757D147C007F527E00BF
:108321001291BAE50F30E64B7B017A0879797F0229
:10833100128C627F8F129A75E50F30E309900879EC
:10834100E04480F08029900875E0FBA3E0FAA3E007
:10835100F9129E3CFF900879E06F6012E92401F95F
:10836100E43AFA129E3CFF90087AE0B50705E490E2
:108371000878F0E4F50EF50F900878E0FF22900BF5
:10838100A0EBF0A3EAF0A3E9F07430129E77900B12
:10839100A0E0FBA3E0FAA3E02401F9E43AFA74783F
:1083A100129E77EF7804A2E713D8FB540FFED39403
:1083B100095005EE2430800574F62E2441FD900B02
:1083C100A0E0FBA3E0FAA3E02402F9E43AFAED12FB
:1083D1009E77EF540FFED394095005EE24308005AB
:1083E10074F62E2441FF900BA0E0FBA3E0FAA3E07A
:1083F1002403F9E43AFAEF129E77900BA0E0FBA375
:10840100E0FAA3E02404F9E43AFAE4029E7790004A
:1084110003E0FD75F002A42412F582E5F0340AF5BB
:1084210083E0FE75F002EDA42411F582E5F0340A33
:10843100F583E0FDEDFF900004E06EF0A3E06FF046
:10844100AFF9EFFEADFAEDFF900004E06EF0A3E0AE
:108451006FF0900003E004F0E0D394054002E4F0F3
:108461009008867490F0E490087CF0A37420F0905A
:108471000004E0FCA3E090087EF0ECA3F09008A0DB
:10848100741DF0A37401F0A37408F0A3747CF0A32D
:108491007404F07B017A0879867D01028F92C0E035
:1084A100C0F0C083C082C0D075D000C000C001C080
:1084B10002C003C004C005C006C0077F0C129B3F69
:1084C1008F0D7F0C129B3F8F13750C00E50D45132B
:1084D100543FF512E50D54C0FF6006E513F45F4209
:1084E1001285120DE51230E51F7F1C129B3F8F0C88
:1084F100E50C541FC394124003430C80E50C541F38
:10850100D394065003430C40E50CFEE512420FEEF6
:10851100420ED007D006D005D004D003D002D0013E
:10852100D000D0D0D082D083D0F0D0E0327BFF7A9F
:10853100A87984123000124800900869EFF0703E6B
:10854100126926900822E07002A3E0700890086981
:108551007409F0802990086D7401F0A3740AF0A3E6
:10856100740AF0900A0EE0900870F0900858E0FB51
:10857100A3E0FAA3E0F91256C5900869EFF0129B47
:10858100E1900957743EF0A37404F0900869E090FB
:108591000959F0900A5EE0FBA3E0FAA3E02401F997
:1085A100E43AFA129E3C900A5DF0A37401F0A374C0
:1085B10009F0A37457F00298BC900B32E064047088
:1085C10061900B36E0FF605A64016056900B38E011
:1085D1007050900B3AE0704A900B3CE07044A3E07D
:1085E1006002803E900B36E064027036900B39E0F9
:1085F1007030900B3BE0FF64816005EF64027022F4
:10860100EFB48121E59620E7FB75960E759701E59C
:108611009620E7FB759611759710900B437403F044
:1086210080031217E3E59620E7FB75960EE4F597B4
:10863100900B42E06404600BE59620E7FB75961110
:1086410075974822900894EFF0E4900896F0FF1295
:108651009744900895EFF0900894E0900AD1F0606B
:108661001F900895E020E066D2B07FC87E00129C82
:1086710066900895E04401F0FDE4FF1299168041EF
:10868100900895E0FF30E046EF54FE900895F0FD2C
:10869100E4FF1299169008977401F0A374F4F09016
:1086A100089774FFF5F0129F3C45F060127F0E129F
:1086B1009744EF30E2097F017E001287DF80E0C23C
:1086C100B0900894E060077F017E001287DF22905E
:1086D1000B32E064026025900B36E0701F900B3A7C
:1086E100E07019A3E07015A3E07011A3E0700D9084
:1086F1000B38E07007A3E0D3940140051217E38023
:1087010044900B39E0D394004031900B327404F063
:10871100E4900B43F0E59620E7FB75960E75970103
:10872100E59620E7FB759612759704E59620E7FB21
:1087310075960EE4F5971257FA800A900B3274037E
:10874100F0900B43F0900B42E06404600BE596203F
:10875100E7FB75961175974822900B32E06404701F
:108761005B900B36E0FF605464016050900B38E081
:10877100704A900B3AE07044900B3CE0703EA3E0ED
:1087810060028038900B36E064027030900B39E063
:10879100702A900B3BE0FF64817021EFB48120E5EA
:1087A1009620E7FB75960E759701E59620E7FB7518
:1087B1009611759740E4900B43F080031217E3E59F
:1087C1009620E7FB75960EE4F597900B42E0640462
:1087D100600BE59620E7FB75961175974822900886
:1087E100AFEEF0A3EFF09008AF74FFF5F0129F3CED
:0E87F10045F060097FE87E03129C6680E92255
:10880000900A0AE0FF900869F064126014E0FE64C8
:1088100014600EEE64156009EE64166004EEB41781
:10882000117B017A0A790B9008B77403F0128DAEB0
:10883000801E900869E0C39480500D900A0AE0FF02
:10884000A3E0FD1299168008900869E0FF129A755E
:10885000900957741BF0A37403F0E4A3F0900A5E30
:10886000E0FBA3E0FAA3E02401F9E43AFA129E3C0B
:10887000900A5DF0A37401F0A37409F0A37457F09B
:108880000298BC900B36E06480701C900B38E0704E
:1088900016A3E07012A3E0700EA3E0700AA3E070CC
:1088A00006A3E0640160051217E38038900B32E004
:1088B000FFB40416900B3374FFF0A374B1F0A374EB
:1088C00086F0900B40E4F0A304F0EFB40316900B95
:1088D0003374FFF0A374B1F0A37488F0900B40E4FC
:1088E000F0A304F0900B42E064046018E59620E7E2
:1088F000FB759611759740900B427401F0E4900B54
:108900003EF0A3F022C0E0C083C082C0D075D0008A
:10891000C000C001C002C003C006C0077821E660E5
:1089200051C2CF08860308E6FA08E62401F9E43AC2
:10893000FA74FF129E55FF7822860308E6FA08E6CD
:10894000F9129E3CFEA807088002C313D8FCFF78EA
:1089500022860308E6FA08E62401F9E43AFA129EB0
:108960003C700B740226F618E436F6782116EF13E5
:108970009293D007D006D003D002D001D000D0D03F
:10898000D082D083D0E032900894EFF07F0212972B
:1089900044900B08E05403FEEF54FC4EFD7F02129E
:1089A00099167F8F129A75750898E47830F6900BB7
:1089B00007E03333335418FF900B0BE0C4335420DB
:1089C0004FFF900B09E025E025E054044FF6900896
:1089D00094E025E0541EFF900B08E0FEC4333354AE
:1089E000C04F08F69008A0741FF0A3E4F0A3740031
:1089F000F0A37430F0A37402F07B007A0079087D54
:108A000001028F927F0A1297449008A3EFF07D2213
:108A10007F011299169008A3E0FD7F0A1299167B38
:108A2000017A0879A47D037F151293EE9008A5E0E2
:108A300054BFF07B017A0879A49008B77403F07FE3
:108A400015128DAEE4FD7F0D129916E4FF129744C6
:108A50009008A3EFF0E4FF1297767F8F129A757F4C
:108A600097129A759008A3E04443F0FDE4FF129931
:108A700016C292D2937F017E001287DFC2A8029DA8
:108A80001E90086974FDF0124800900869EFF070BC
:108A900029900A12E0FD90086E7401F0A3740AF0A8
:108AA000A37414F0900A13E0900871F07B017A0A25
:108AB000790A12538C900869EFF0129BE1900957E4
:108AC0007448F0A37403F0900869E0FF3395E0FE6A
:108AD0007CFF7DFF129E89900959EFF07B017A0996
:108AE0007957900A5EEBF0A3EAF0A3E9F02401F9CC
:108AF000E43AFA129E3C900A5DF00298BC900B9307
:108B0000EBF0A3EAF0A3E9F0129CCC900B97EFF006
:108B1000900B967433F0C2A89008BCE4F0A3F0A3C5
:108B2000F0A3F0A3F0A304F0FB7A0B7996FD128B6F
:108B3000EC9008BCE4F0A3F0A3F0A3F0A3F0A3F042
:108B40007B017A0B79977D01128BEC900B93E0FB04
:108B5000A3E0FAA3E02401F9E43AFA9008BCE4F0B7
:108B6000A3F0A3F0A3F0A37402F0E4A3F07DFB1242
:108B70008BECD2A8227B017A0A790C90087CEBF06E
:108B8000A3EAF0A3E9F0E4FF129E3C703B90087C5E
:108B9000E0FBA3E0FAA3E02401F9E43AFA129E3CD8
:108BA000702690087CA3E0FAA3E02402F9E43AFAE4
:108BB000129E3C701390087CA3E0FAA3E02403F912
:108BC000E43AFA129E3C602390087CE0F9A3E0FAB4
:108BD000A3E0900882C9F0A3EAF0A3E9F090085856
:108BE000E0FBA3E0FAA3E0F9125DFB229008B8EBEA
:108BF000F0A3EAF0A3E9F09008C1E06002C294E4B7
:108C0000FFEFC39D50259008B8E0FBA3E0FAA3E076
:108C10002FF9E43AFA129E3CF5A3E5F830E7FB752C
:108C2000F8019008C2E5A3F00F80D6E4FF9008BFDA
:108C3000E0FEEFC39E5022E4F5A3E5F830E7FB75B4
:108C4000F8019008BCE0FBA3E0FAA3E02FF9E43AB6
:108C5000FAE5A3129E770F80D49008C0E06002D29C
:108C600094229008A6EFF0A3EBF0A3EAF0A3E9F0BA
:108C7000A3745EF0C2A89008BC7401F0A37408F05D
:108C8000A374AAF0A37401F0E4A3F0A304F0FB7AA8
:108C90000879AAFD128BEC9008AA747FF09008A7BF
:108CA000E0F9A3E0FAA3E09008BCC9F0A3EAF0A3BE
:108CB000E9F09008A6E09008BFF0A37402F0E4A3E6
:108CC000F07B017A0879AA7D01128BECD2A8229060
:108CD0000B32E064047024900B36E06481701C90C9
:108CE0000B38E07016A3E07012A3E0700EA3E070E2
:108CF0000AA3E07006A3E0640160051217E3801682
:108D0000900B3374FFF0A374B1F0A37488F0900B50
:108D100040E4F0A304F0900B42E064046018E59690
:108D200020E7FB759611759740900B427401F0E4B3
:108D3000900B3EF0A3F02290088CEFF0D2937F01CD
:108D40007E001287DF12797190088DEFF03395E085
:108D5000FEEF25E0FFEE33FE746D2FF9740A3EFA44
:108D60007B0190088CE0FD124E0690088DE02FF0FC
:108D70007B017A08798C7D017C001281C3AD07AC40
:108D80000690088D12906090088DE02FF07B017A9C
:108D90000A796DE0FD3395E0FC1298E7D29322F05A
:108DA0007A0879A87B019008B77403F07F149008C3
:108DB000B3EFF0A3EBF0A3EAF0A3E9F09008B3E07F
:108DC0004420F0C2A89008BCE4F0A3F0A3F0A3F004
:108DD000A3F0A304F0FB7A0879B3FD128BEC9008A2
:108DE000B7E0FD9008BCE4F0A3F0A3F0A3F0A374F7
:108DF00002F0E4A3F09008B4E0FBA3E0FAA3E0F9EA
:108E0000128BECD2A8229008707401F0A37401F0C8
:108E1000A3741AF0E4FFFEFD8047E47F087E07FD9F
:108E2000FC90086CE0F8A3E0F9A3E0FAA3E0FBC330
:108E300012A0CF5035900870E0FBA3E475F001124A
:108E40009F3CA9F0FAE4129E7790086CE0FCA3E046
:108E5000FDA3E0FEA3E02401FFE43EFEE43DFDE4CB
:108E60003CFC90086C12A10680B022900894EBF0B4
:108E7000A3EAF0A3E9F0E4A3F07F80FE1298317F2B
:108E80008F129A757F5F7E00129831E50F20E023E4
:108E9000E50F541E600890089774FFF08026900834
:108EA00094E0FBA3E0FAA3E0F9124000900897EFEA
:108EB000F08011900894E0FBA3E0FAA3E0F9E4F558
:108EC000F0129F7D7F8F129A75900897E0FF22E441
:108ED000900869F07F0512974490086A129740EF56
:108EE00030E211900869E024B8F0EF30E020E0248F
:108EF00005F0801A900869E024BEF0EF30E004E04D
:108F00002408F0EF30E107900869E024F6F0EFC4A0
:108F10001313540375F003A4FF90086AE0900869E6
:108F200030E706E0C39FF08003E02FF0900869E08F
:108F3000FF22E0FBA3E0FAA3E0F99008C7EFF0906E
:108F400008CAEBF0A3EAF0A3E9F09008C8ECF0A39C
:108F5000EDF04C603C9008C7E0F5964396C0E4FF06
:108F6000FED39008C9E09F9008C8E09E4020E59697
:108F700020E7FB9008CAE0FBA3E0FAA3E02FF9EAA0
:108F80003EFAE597129E770FBF00010E80D3E4F5FD
:108F900096229008A0E04420F0C2A89008BCE4F01B
:108FA000A3F0A3F0A3F0A3F0A304F0128BEC9008BD
:108FB000BCE4F0A3F0A3F0A3F0A3F0A3F07B017A4C
:108FC0000879A07D01128BEC9008A4E0FD9008BC0C
:108FD000E4F0A3F0A3F0A3F0A37402F0E4A3F090F4
:108FE00008A1E0FBA3E0FAA3E0F9128BECD2A822DF
:0F8FF000E4FFFE0FBF00010EBE01F8BFF4F52233
:10900000900A5CE0703204F09008CAF0A3740AF091
:10901000A37408F0900A49E0FBA3E0FAA3E024015E
:10902000F9E43AFA129E3C049008CDF0900A49A364
:10903000E0FAA3E0F9023FBF900A49E0FBA3E0FA9F
:10904000A3E0F9129E3C9008CAF0900A08E090084C
:10905000CBF07BFF7AA879BF12300022AD07AC06B7
:10906000E0FF3395E0FEEF25E0FFEE33FE746D2F59
:10907000F9740A3EFA7B019008A3EBF0A3EAF0A38F
:10908000E9F0A3ECF0A3EDF0F4FFECF4FE9008A6F9
:10909000F0A3EFF0EEFD124E069008A4E475F00484
:1090A000129F269008A3E0FBA3E0FAA3E0F9A3A394
:1090B000E0FD124E067F0422900B7DEFF0900B80B6
:1090C000EBF0A3EAF0A3E9F0900B7EECF0A3EDF057
:1090D0004C603BE59620E7FB900B7DE0F596E4FFC6
:1090E000FED3900B7FE09F900B7EE09E4020900B84
:1090F00080E0FBA3E0FAA3E02FF9EA3EFA129E3CDF
:10910000F597E59620E7FB0FBF00010E80D3229074
:1091100008C7EFF09008CAEBF0A3EAF0A3E9F090DB
:1091200008C8ECF0A3EDF04C603BE59620E7FB901F
:1091300008C7E0F596E4FFFED39008C9E09F9008C9
:10914000C8E09E40209008CAE0FBA3E0FAA3E02F0D
:10915000F9EA3EFA129E3CF597E59620E7FB0FBF31
:1091600000010E80D322C0E0C083C082C0D075D081
:1091700000C000C001C002C003C2997916E778158B
:10918000667005781BF680187817860308E6FA08DB
:10919000E6F97816E60629F9E43AFA129E3CF599C2
:1091A00030980678147601C298D003D002D001D04E
:1091B00000D0D0D082D083D0E03290089CEEF0A3D3
:1091C000EFF0A3ECF0A3EDF090089CE0550EFEA3A9
:1091D000E0550F4E7024A3E07002A3E0601CE591FF
:1091E00030E7E57FE87E031297DB90089FE024FFDD
:1091F000F090089EE034FFF080CE90089EE0700270
:10920000A3E07009129C2D750E00750F0122900BC2
:1092100036E0701D900B3AE07017A3E07013A3E0E6
:10922000700FA3E0700B900B38E07005A3E030E7FF
:10923000031217E3900B427405F0900B39E0900B8A
:109240003260057403F080037402F0900B42E06416
:1092500004600BE59620E7FB759611759748229000
:109260000A0AE0600EA3E0B4FF047F018002E4FF7D
:10927000128645900A0DE06006A3E0FF126C77901D
:1092800009577419F0A3740EF0E4A3F0A3F0A3F04F
:10929000A3F0128ECF90095DEFF0900A5D740EF08E
:1092A000A37401F0A37409F0A37457F00298BC12E0
:1092B0007FFAEF603CE490085CF0900A08E0645D9F
:1092C0006003125F61900A08E075F003A42486F53C
:1092D00082E5F034ACF583E4740193FA740293F9F7
:1092E00012A158900854E07003129CC6E4900854F0
:1092F000F090085CE060057F01129BCF2274022F82
:10930000F58274093EF583E0FF9009A3E0600BE469
:10931000F09009A2F0781BE670FB9009A2E024A46B
:10932000F582E43409F583EFF09009A2E004F0E05F
:10933000FDC394645004EFB40A0F7B017A0979A449
:109340001297AA9009A37401F0229008C7EFF0E4E5
:10935000A3F09008C8E0FFD394035039EF25E0252F
:10936000E02461F582E4340AF583E0FF9008C7E069
:10937000FEEFB50618A3E025E025E02462F582E4BF
:10938000340AF583A3E0FAA3E0F902A1589008C8D3
:10939000E004F080BD22900A09E064047043900963
:1093A000577456F0A37403F07B017A097957900A39
:1093B0005EEBF0A3EAF0A3E9F02401F9E43AFA1233
:1093C0009E3C900A5DF09009597401F01298BC7FA0
:1093D000647E001287DFE4FDFF7E1012986275EF55
:1093E0001022EFF07A08797E7B017D037F149008CC
:1093F000B3EFF0A3EBF0A3EAF0A3E9F0C2A8900862
:10940000B3E04460F0A3E0F9A3E0FAA3E09008BC65
:10941000C9F0A3EAF0A3E9F0A3EDF0A37402F0A36E
:1094200014F0FB7A0879B3FD128BECD2A822E596F2
:1094300020E7FB759601759708E59620E7FB759682
:1094400007759707E59620E7FB759609759707E579
:109450009620E7FB75960B75970775D7E0E5962084
:10946000E7FB75960F75978043E602D2AFE596202D
:10947000E7FB75960175970122900B39E0FF129377
:109480004A900A5EE0F9A3E0FAA3E0900B33C9F03A
:10949000A3EAF0A3E9F0900A5DE0FF900B40E4F04E
:1094A000A3EFF0900B42E064046018E59620E7FB20
:1094B000759611759740900B427401F0E4900B3E45
:1094C000F0A3F022E4F50EF50F7D03FF129916C20A
:1094D00092D293129D217B017A0879B07D037F158A
:1094E0001293EE9008B1E04440F07B017A0879B025
:1094F0009008B77403F07F15128DAE7F0C1297445D
:10950000E4F50EF50F7D3F7F0D129916D2A82212B9
:10951000102F900A49E0F9A3E0FAA3E0900B33C9B9
:10952000F0A3EAF0A3E9F0900B3CE0FFA3E0900B7E
:1095300040CFF0A3EFF0900B42E064046018E59692
:1095400020E7FB759611759740900B427402F0E48A
:10955000900B3EF0A3F02290086BEFF090085BE0D8
:10956000FE6F6031EE24FE60080470081267FF8011
:1095700003129D1890086BE024FE600E04700E7BB1
:10958000017A08794F129D1B8003129CB790086BDB
:10959000E090085BF022E4900869F0129BE19009EA
:1095A00057744CF0A37440F0900869E0900959F0AA
:1095B000A3740AF07B017A097957900A5EEBF0A355
:1095C000EAF0A3E9F02401F9E43AFA129E3C900A89
:1095D0005DF00298BCE4900869F0129BE190095795
:1095E0007450F0A37440F0900869E0900959F0A31A
:1095F000740AF07B017A097957900A5EEBF0A3EACE
:10960000F0A3E9F02401F9E43AFA129E3C900A5DD5
:10961000F00298BCD2937F067E001287DF9008820A
:1096200074AAF0900884F0900886740AF090088379
:109630007408F0900885F09008877404F07B017A34
:109640000879827D037C001298E7D2937F017E0027
:109650000287DFE47814F6781BF67815F608F690A2
:1096600009A3F09009A2F0C29FD29DD29C758840B8
:10967000758920438E08758D30D28E43A41075E114
:109680000175B283D2BC75A890D2ACD2AF43E24090
:1096900022900B36E06401701C900B3CE07016A326
:1096A000E07012900B38E0700CA3E07008A3E0703B
:1096B00004A3E060031217E3900B42E06404600B24
:1096C000E59620E7FB7596117597482274FF900880
:1096D00069F0A3F0EE3395E0FDFCE47B30FAF9F895
:1096E000129F9CC374FF9F90086AF074FF9E9008BD
:1096F00069F0E4F5C8438E30E0FEA3E0FDF5CA8DC5
:10970000CCEEF5CBF5CD2243A40443A701D282C20F
:10971000B075A16075A20B75F801129C4643A405B3
:1097200043A60675A51FD2A043E10243E2C0C29042
:10973000D291D294C2A17F647E00129C66D2A122F3
:10974000EFF07F0A9008B3EFF0C2A8E04440F09039
:1097500008BC7401F0A37408F0A374B4F0A37401FE
:10976000F0A3F0A3F0FB7A0879B3FD128BECD2A83A
:109770009008B4E0FF229008A7EFF070077D407FCB
:10978000091299169008A7E0B406077D807F091298
:1097900099167F03129744EF540FFF9008A7E0FE3D
:1097A000C454F04FFD7F03029916E490090FF0783E
:1097B0001BE670FB781B76017817A60308A6020843
:1097C000A60178167601AF0518A607781786030854
:1097D000E6FA08E6F9129E3CF599227C007D041217
:1097E000A15EC374FF9FFF74FF9EFC538EBFE4F520
:1097F00091EFFBF592ECF5938B94F5954391042250
:109800007E007F407D007B017A09795712A3359055
:109810000957745CF0A37440F0E4A3F0900A5D74FF
:1098200040F0A37401F0A37409F0A37457F00298F8
:10983000BC8E108F11E4FFFEE50E5510FCE50F55B0
:10984000114C700B0FBF00010EBEFFECBFFDE9D342
:10985000EF94F0EE94FF4009129C2D750E00750FE9
:109860000122A2AF9201C2AF75FF8075EF028E1088
:109870008F1175B7A575B7F1438F0175FF8075EF2F
:1098800002851182851083EDF0538FFEA20192AF05
:10989000229009577405F0900955E0900958F0900E
:1098A0000956E0900959F0900A5E7401F0A374091A
:1098B000F0A37457F0900A5D7403F022E490087CE2
:1098C000F0900958E0FF90087CE0FEC39F501774A9
:1098D000572EF582E43409F583E0FF129C3A900894
:1098E0007CE004F080DB227822A60308A60208A60A
:1098F00001E408F6AF057821A60775C804AFA8757E
:10990000A820D2AF7821E670FB30CFFD8FA8E4F518
:10991000C822E0FDE4FF9008B3EFF0A3EDF0C2A889
:109920009008BCE4F0A3F0A3F0A3F0A304F0A3F02C
:10993000FB7A0879B37D02128BECD2A822129968C7
:10994000EF3395E0FEEF2480FFE43EAB07FA7C00A6
:109950007D0CFE129E89AC06AD07EAC313FEEB1325
:109960002DFBEC3EFEAF03227F87129A757F147E9B
:1099700000129C667F19129744EF5480FD3395E0E6
:109980004D6006EF547FFE8006EF547FF404FEAF77
:109990000622900B9DEBF0A3EAF0A3E9F0900B9D5B
:1099A000E0FBA3E0FAA3E0F912A901AD07900B9D3B
:1099B000E0FBA3E0FAA3E0F90297AA90084BE0705D
:1099C00002A3E070037F0122129BA9C390084CE020
:1099D0009F90084BE09E500990084E7401F07F0064
:1099E000227F01227F96129A757F97129A757FF4D3
:1099F0007E01129C667F0F129744900892EFF07FD1
:109A000096129A75900892E0FF22438E045388EFD5
:109A100053D8BFE58954F04401F589E4F58AF58C03
:109A200075D90475D840F5F9F5FA43881022C29427
:109A30008FA3E5F830E7FB75F801E5A3129E77E404
:109A4000F5A3E5F830E7FB75F801E5A3129E77D2A0
:109A500094229009597402F09009577415F0A37478
:109A600003F0900A5DF0A37401F0A37409F0A374ED
:109A700057F00298BC9008A7EFF0C2A89008BCE489
:109A8000F0A3F0A3F0A3F0A304F0A3F0FB7A08790D
:109A9000A7FD128BECD2A822900BA6EFF0A3EDF05D
:109AA0009008BCE4F0A3F0A3F0A3F0A3F0A304F0AB
:109AB000FB7A0B79A67D02028BEC43B203E4F5B985
:109AC00043B980128FF043B9C0128FF0E5B930E589
:109AD000FB75B69075A90322E4FF129744EF30E7B7
:109AE00013EF547FFDE4FF1299167F017E00128769
:109AF000DF1270002275F003EFA42486F582E5F0F2
:109B000034ACF583740193FA740293F902A158906E
:109B10000A49E0FBA3E0FAA3E02401F9E43AFA12CF
:109B20009E3C9009A0F022C2A89008BCE4F0A3F0EB
:109B3000A3F0A3F0A304F0A3F0128BECD2A822C2EE
:109B4000A8EF4440FF7B017A097910129A2ED2A81F
:109B5000900910E0FF22EF30E7028009EF547FFF09
:109B6000C3747F9FFFAD077F180299167F18129765
:109B700044EF30E7028009EF547FFFC3747F9FFFFB
:109B800022900B42E06404600BE59620E7FB75969B
:109B90001175974822900AD2E0FD7F051299169020
:109BA0000AD3E0FD7F0A029916AFFA7E00ADF97C78
:109BB00000ABFAEBB507F2EFFEEDFF22E4FF1297E0
:109BC00044EF20E709EF4480FDE4FF1299162212CA
:109BD0004C181298BC7F02900959E06003B401EF61
:109BE00022129A0AE4FF12864590085CE070031284
:109BF0007A27229008C7E004F070069008C6E004B7
:109C0000F0229008C7E004F070069008C6E004F067
:109C1000229001197401F0900A0AE0FF029BCFE440
:109C200090085BF0A3F0900854F0027A27127A278C
:109C30007F017E001287DF025F61781BE670FB7890
:109C40001B76018F9922D28375E40BD288D2A8D2D9
:109C5000AF227814E670FBE47814F6227F0D7E00C4
:109C60001296CC7F00221297DBE59130E7FB227F32
:109C700002129557026F7C7F02129557028A817FEC
:109C8000011295570268007F0112955702739C7F5D
:109C9000011295570265107F0112955702663F7FAA
:109CA0000112955702852E7F011295570246E37FD8
:109CB000011295570263DFE4FF1297767F0022E4DA
:109CC0007814F6AF9922E4900A5CF0227F13129781
:109CD0004422E47814F6227F15028D377F0A028D24
:109CE000377F09028D377F08028D377F02028C6231
:109CF0007F9D029A757F80029A757F01227F0022E4
:109D0000025FFF0276A402925F02880002812E02A7
:109D10007CEB0282587F00227F00220244B4C2946E
:109D200022D29422E709F608DFFA8046E709F20812
:109D3000DFFA803E88828C83E709F0A3DFFA803265
:109D4000E309F608DFFA8078E309F208DFFA8070A9
:109D500088828C83E309F0A3DFFA806489828A8396
:109D6000E0A3F608DFFA805889828A83E0A3F2082C
:109D7000DFFA804C80D280FA80C680D4806980F27D
:109D80008033801080A680EA809A80A880DA80E202
:109D900080CA803389828A83ECFAE493A3C8C5829F
:109DA000C8CCC583CCF0A3C8C582C8CCC583CCDFE2
:109DB000E9DEE7800D89828A83E493A3F608DFF960
:109DC000ECFAA9F0EDFB2289828A83ECFAE0A3C8C1
:109DD000C582C8CCC583CCF0A3C8C582C8CCC58316
:109DE000CCDFEADEE880DB89828A83E493A3F20891
:109DF000DFF980CC88F0EF60010E4E60C388F0ED93
:109E00002402B4040050B9F582EB2402B4040050DB
:109E1000AF2323458223909D7473C2D530F707B2D8
:109E2000D563F0FF05F030E70CB2D5F4048463F09D
:109E3000FF05F080018430D502F40422BB010689BD
:109E4000828A83E0225002E722BBFE02E32289825B
:109E50008A83E49322BB010989828A83F8E028F08F
:109E600022500327F722BBFE05F8E328F3228A835A
:109E70008982F8E4932822BB010689828A83F02232
:109E80005002F722BBFE01F322EF8DF0A4A8F0CF21
:109E90008CF0A428CE8DF0A42EFE22BC000BBE00B8
:109EA00029EF8DF084FFADF022E4CCF875F008EFD7
:109EB0002FFFEE33FEEC33FCEE9DEC984005FCEEFC
:109EC0009DFE0FD5F0E9E4CEFD22EDF8F5F0EE842D
:109ED00020D21CFEADF075F008EF2FFFED33FD40F2
:109EE00007985006D5F0F222C398FD0FD5F0EA226C
:109EF000C2D5EC30E709B2D5E4C39DFDE49CFCEE8D
:109F000030E715B2D5E4C39FFFE49EFE129E9BC3CB
:109F1000E49DFDE49CFC8003129E9B30D507C3E4C6
:109F20009FFFE49EFE22C5F0F8A3E028F0C5F0F8FC
:109F3000E582158270021583E038F022A3F8E0C5AF
:109F4000F025F0F0E582158270021583E0C838F044
:109F5000E822BB010A89828A83E0F5F0A3E022505F
:109F60000687F009E71922BBFE07E3F5F009E319BC
:109F70002289828A83E493F5F074019322BB010A5B
:109F800089828A83F0E5F0A3F0225006F709A7F052
:109F90001922BBFE06F3E5F009F31922E88FF0A4BD
:109FA000CC8BF0A42CFCE98EF0A42CFC8AF0EDA460
:109FB0002CFCEA8EF0A4CDA8F08BF0A42DCC382593
:109FC000F0FDE98FF0A42CCD35F0FCEB8EF0A4FE73
:109FD000A9F0EB8FF0A4CFC5F02ECD39FEE43CFC08
:109FE000EAA42DCE35F0FDE43CFC2275F008758224
:109FF00000EF2FFFEE33FECD33CDCC33CCC5823313
:10A00000C5829BED9AEC99E58298400CF582EE9B17
:10A01000FEED9AFDEC99FC0FD5F0D6E4CEFBE4CD35
:10A02000FAE4CCF9A88222B800C1B90059BA002DCF
:10A03000EC8BF084CFCECDFCE5F0CBF97818EF2F88
:10A04000FFEE33FEED33FDEC33FCEB33FB10D703B7
:10A05000994004EB99FB0FD8E5E4F9FA227818EF60
:10A060002FFFEE33FEED33FDEC33FCC933C910D7BF
:10A07000059BE99A4007EC9BFCE99AF90FD8E0E4CC
:10A08000C9FAE4CCFB2275F010EF2FFFEE33FEEDA2
:10A0900033FDCC33CCC833C810D7079BEC9AE89972
:10A0A000400AED9BFDEC9AFCE899F80FD5F0DAE454
:10A0B000CDFBE4CCFAE4C8F922EB9FF5F0EA9E422E
:10A0C000F0E99D42F0EC6480C864809845F022EB92
:10A0D0009FF5F0EA9E42F0E99D42F0E89C45F022AF
:10A0E000E8600FECC313FCED13FDEE13FEEF13FF5E
:10A0F000D8F122E8600FEFC333FFEE33FEED33FDFE
:10A10000EC33FCD8F122ECF0A3EDF0A3EEF0A3EFDA
:10A11000F022BB010789828A8302A36A5005E9F80D
:10A1200002A361BBFE05E9F802A37389828A830258
:10A13000A37CD083D082F8E4937012740193700DE5
:10A14000A3A393F8740193F5828883E47374029354
:10A150006860EFA3A3A380DF8A838982E473EC8E17
:10A16000F0A4CCC5F0CCCDF8EFA4CEC5F02DFDE425
:10A170003CFCE8A42EC8C5F03DFDE43CFCEFA4FF88
:10A18000E5F028FEE43DFDE43CFC22E3F5F009E2C5
:10A1900008B5F06BDFF58067E3F5F009E608B5F088
:10A1A0005EDFF5805A87F009E608B5F052DFF680E9
:10A1B0004E87F009E208B5F046DFF6804288828CCF
:10A1C0008387F009E0A3B5F036DFF6803288828C11
:10A1D0008387F009E493A3B5F025DFF58021888219
:10A1E0008C83E3F5F009E0A3B5F014DFF580108867
:10A1F000828C83E3F5F009E493A3B5F002DFF40267
:10A20000A2BA808780E9809080D4803E8015806EDD
:10A21000807E809D80B7808D80A380518074803C3B
:10A2200002A2C689828A83ECFAE493F5F0A3C8C53A
:10A2300082C8CCC583CCE493A3C8C582C8CCC583EF
:10A24000CCB5F076DFE3DEE1807089828A83E49327
:10A25000F5F0A3E208B5F062DFF4805E89828A83BC
:10A26000E0F5F0A3E608B5F051DFF5804D89828A6C
:10A2700083E0F5F0A3E208B5F040DFF5803C898289
:10A280008A83E493F5F0A3E608B5F02EDFF4802A84
:10A290008002805789828A83ECFAE493F5F0A3C8A0
:10A2A000C582C8CCC583CCE0A3C8C582C8CCC58351
:10A2B000CCB5F006DFE4DEE280007FFFB5F0020FF0
:10A2C0002240027F012289828A83ECFAE0F5F0A322
:10A2D000C8C582C8CCC583CCE0A3C8C582C8CCC5DC
:10A2E00083CCB5F0D5DFE5DEE380CF89828A83ECCD
:10A2F000FAE0F5F0A3C8C582C8CCC583CCE493A32B
:10A30000C8C582C8CCC583CCB5F0AFDFE4DEE2803F
:10A31000A988F0EF60010E4E60ABED2402B404009A
:10A320005098F582EB2402B40400508E232345821A
:10A330002390A20273EF4E6012EF60010EEDBB019D
:10A340000B89828A83F0A3DFFCDEFA2289F05007B2
:10A35000F709DFFCA9F022BBFEFCF309DFFCA9F042
:10A3600022E6FB08E6FA08E6F922E0FBA3E0FAA3FE
:10A37000E0F922E2FB08E2FA08E2F922E493FB7436
:10A380000193FA740293F922726561642072656721
:10A39000733A2025686878202568687820256868E1
:10A3A0007820256868780A00454E2070696E20661E
:10A3B00061696C65640A004952512070696E202FF2
:10A3C0002072656164696E672049525120666C6134
:10A3D0006773206661696C65640A0043616E6E6F25
:10A3E000742072756E206F6E204153333939300AF4
:10A3F0000043616E6E6F742072756E206F6E204127
:10A4000053333939310A00556E6B6E6F776E2063A6
:10A4100068697020256868780A000A7265672025D7
:10A420006868782020200025686878200025686802
:10A43000780000000102030405060708090A0B0C56
:10A440000D0E0F101112131415161718191A1B1CC4
:10A450001D1E1F202122232425262728292A2B2CB4
:10A460002D2E2F303132333435363738393A3B3CA4
:10A470003D3E3F404142434445464748494A4B4C94
:10A480004D4E4F505152535455565758595A5B5C84
:10A490005D5E5F606162636465666768696A6B6C74
:10A4A0006D6E6F707172737475767778797A7B7C64
:10A4B0007D7E7F808182838485868788898A8B8C54
:10A4C0008D8E8F909192939495969798999A9B9C44
:10A4D0009D9E9FA0A1A2A3A4A5A6A7A8A9AAABAC34
:10A4E000ADAEAFB0B1B2B3B4B5B6B7B8B9BABBBC24
:10A4F000BDBEBFC0C1C2C3C4C5C6C7C8C9CACBCC14
:10A50000CDCECFD0D1D2D3D4D5D6D7D8D9DADBDC03
:10A51000DDDEDFE0E1E2E3E4E5E6E7E8E9EAEBECF3
:10A52000EDEEEFF0F1F2F3F4F5F6F7F8F9FA011ABF
:10A5300000011400011B01500B57BFAFA7A3A1A03E
:10A54000B0B8BCBE41888A642082490B455580C0A2
:10A55000E0F0F8FCFEFF490B4EFF7F3F1F0F0703A3
:10A560000100480998FFFFFFFFFFFFFFFF60400960
:10A5700015000000000000000000000000000000C6
:10A5800000000000000000000000000000000000CB
:10A5900000000000000000000000000000000000BB
:10A5A00000000000000000000000000000000000AB
:10A5B00000490B67FFAC65FFAC6AFFAC76430B420A
:10A5C0000003034C0A6105FF9891000000000000A1
:10A5D0000000500A4C02FF9B0F000000000000002A
:10A5E0000000000000410A5C0045084F0C0200001A
:10A5F0000141085704410862034108613244085D83
:10A60000000DC65E44000B000E26124208460000F4
:10A610004208240190420855000041085C004108AE
:10A620004D024100000041000100410002004100D4
:10A630000300420B0C000A010D00010C00020E0089
:10A6400000410AD100420AEFBB80410AF1000066D6
:10A650006F756E64207769746820706F77536C6FC4
:10A66000743D2568687820257820746167732C20F4
:10A670006D617820256868780A002D002E0020255D
:10A680006868780A002048656C6C6F20576F726CA0
:10A6900064210A204D79206E616D65206973204D1B
:10A6A0004952434F210A2057656C636F6D652074D2
:10A6B0006F20766973697420726669642E656C65B3
:10A6C000636B6974732E636F6D0A0061733339397C
:10A6D00078496E697469616C697A652829207265A8
:10A6E0007475726E65642025780A005072696E7404
:10A6F000205043202568687820256868780A005033
:10A7000072696E74204550432000256868782000E7
:10A710000A0054414720256868783A0A00524E31B1
:10A72000363A202568687820256868780A004E75D2
:10A730006D626572206F6620726561642062797453
:10A7400065733A2025640A0050433A2025686878EA
:10A750002025686878004550433A20004550434C16
:10A76000454E20286279746573293A20256868640B
:10A770000A0048414E444C453A2025686878202517
:10A780006868780A000000787FE4F6D8FD75817F5C
:10A7900075D90002A7D1022000E493A3F8E493A3A3
:10A7A0004003F68001F208DFF48029E493A3F85413
:10A7B00007240CC8C333C4540F4420C8834004F496
:10A7C00056800146F6DFE4800B01020408102040A9
:10A7D0008090A52EE47E019360BCA3FF543F30E53A
:10A7E00009541FFEE493A360010ECF54C025E0601E
:10A7F000A840B8E493A3FAE493A3F8E493A3C8C5EC
:10A8000082C8CAC583CAF0A3C8C582C8CAC583CADC
:10A81000DFE9DEE780BE63617574696F6E20777271
:10A820006F6E6720636869700A00415333393932AB
:10A8300020526561646572204669726D7761726548
:10A8400020322E322E390A00415333393932204515
:10A850006C65636B69747320436F6C7420616E6404
:10A86000204D4943524F20312E320A0057726F6EED
:10A87000672076657273696F6E20747970652073D6
:10A88000656E64004B494C4C205461670A00256892
:10A8900068782025686878202568687820256868A9
:10A8A0007820256868782025686878202568687889
:10A8B00020256868780A002568687820000A0075F5
:10A8C0007362206572726F72202D207265706F72D4
:10A8D000742025686878206C6F73742061667465D5
:10A8E0007220256868780A000A0A53656E64506110
:10A8F000636B65742074696D6564206F75740A0AF2
:10A9000000E4FFFE129E3C600C0FEF70010E09E99F
:10A9100070F20A80EF22120110010000004025139E
:10A9200029C0000001020001090229000101008084
:10A93000AF09040000020300000009210101000129
:10A9400022140307058103400001070502034000AC
:10A95000010600FF0901A10185109502750826FF77
:10A960000015000901910285119530750826FF0038
:10A9700015000901810285319502750826FF001531
:10A9800000090191028532953F750826FF001500E8
:10A99000090181028533953F750826FF00150009DE
:10A9A00001910285349502750826FF001500090102
:10A9B00081028514953D750826FF00150009019157
:10A9C0000285159502750826FF0015000901810210
:10A9D0008518950D750826FF00150009019102855F
:10A9E00019950D750826FF001500090181028535AE
:10A9F000953F750826FF00150009019102853695DF
:10AA000003750826FF0015000901810285379507A7
:10AA1000750826FF001500090191028538953F75DC
:10AA20000826FF00150009018102851C95027508A2
:10AA300026FF00150009019102851D950575082660
:10AA4000FF00150009018102851A9505750826FF8A
:10AA500000150009019102851B9502750826FF006B
:10AA6000150009018102853F950C750826FF001528
:10AA700000090191028540950F750826FF00150019
:10AA8000090181028547953F750826FF00150009D9
:10AA900001910285489502750826FF0015000901FD
:10AAA00081028549950C750826FF00150009019162
:10AAB00002854A953F750826FF00150009018102AD
:10AAC000854B953F750826FF001500090191028509
:10AAD0004C953F750826FF00150009018102854D40
:10AAE000953F750826FF00150009019102854E95D6
:10AAF0003F750826FF00150009018102854F953F2B
:10AB0000750826FF001500090191028550953F75D3
:10AB10000826FF001500090181028541953F75084F
:10AB200026FF001500090191028542953F75082610
:10AB3000FF0015000901810285439502750826FF73
:10AB4000001500090191028544953F750826FF0014
:10AB5000150009018102853B9507750826FF001540
:10AB60000009019102853E9502750826FF00150037
:10AB700009018102853D9506750826FF001500092B
:10AB8000019102853C9502750826FF001500090118
:10AB9000810285459509750826FF00150009019178
:10ABA0000285469504750826FF00150009018102FB
:10ABB0008555953F750826FF00150009019102850E
:10ABC000569502750826FF00150009018102855877
:10ABD000953F750826FF00150009018102855795EC
:10ABE00001750826FF00150009019102855A953F5D
:10ABF000750826FF001500090181028559953F75EA
:10AC00000826FF00150009019102855C953F750833
:10AC100026FF00150009018102855B953F75082616
:10AC2000FF00150009019102855E953F750826FF1A
:10AC300000150009018102855D9503750826FF0056
:10AC40001500090191028560953F750826FF0015E2
:10AC50000009018102855F953F750826FF001500F8
:10AC600009019102C005030904000A0361006D0097
:10AC70007300200000000E03410053003300390030
:10AC8000390078000000FF9D00FF9D00FF9D00FF40
:10AC90009D00FF9D00FF9D00FF9D00FF9D00FF9D0B
:10ACA00000FF9D00FF9D00FF9D00FF9D00FF9D0098
:10ACB000FF9D00FF9D00FF9D03FF9D00FF9D00FF86
:10ACC0009D00FF9A52FF9D00FF9D00FF9D00FF9D8C
:10ACD00006FF9D00FF9D09FF9D00FF9D0CFF9D004D
:10ACE000FF9D00FF9D00FF9D00FF9D00FF9D00FF59
:10ACF0009D00FF9D00FF9D00FF9D00FF9D00FF9DAB
:10AD000000FF9D00FF9D00FF9D00FF9D00FF9D0037
:10AD1000FF9D00FF9D00FF9D00FF2FEAFF9D00FFAC
:10AD20009C7FFF9D00FF9C87FF9D00FF9C8FFF9DE8
:10AD300000FF9D00FF9D00FF9C97FF9D00FF9C9FD3
:10AD4000FF9D00FF51CFFF9D00FF1800FF9D00FFFA
:10AD50009C11FF9D00FF9CA7FF9D00FF9C77FF9D1E
:10AD600000FF9C6FFF9D00FF9596FF9D00FF7E47B3
:10AD7000FF9D00FF95D5FF9D00FF9D00FF9D00FFFB
:10AD80009D00FF9D00FF9396FF9D00FF9D12FF9D7C
:10AD900000FF9D0FFF9D00FF9800FF9D00FF4FB932
:10ADA000FF9D00FF9CAFFF9D00FF9D00FF9D00FFEA
:10ADB0009D00FF9D00FF9D00FF9D00FF9D00FF9DEA
:10ADC00000FF9D00FF9D00FF9D00FF9D00FF9D0077
:10ADD000FF9D00FF9D00FF9D00FF9D00FF9D00FF68
:10ADE0009D00FF9D00FF9D00FF9D00FF9D00FF9DBA
:10ADF00000FF9D00FF9D00FF9D00FF9D00FF9D0047
:10AE0000FF9D00FF9D00FF9D00FF9D00FF9D00FF37
:10AE10009D00FF9D00FF9D00FF9D00FF9D00FF9D89
:10AE200000FF9D00FF9D00FF9D00FF9D00FF9D0016
:10AE3000FF9D00FF9D00FF9D00FF9D00FF9D00FF07
:10AE40009D00FF9D00FF9D00FF9D00FF9D00FF9D59
:10AE500000FF9D00FF9D00FF9D00FF9D00FF9D00E6
:10AE6000FF9D00FF9D00FF9D00FF9D00FF9D00FFD7
:10AE70009D00FF9D00FF9D00FF9D00FF9D00FF9D29
:10AE800000FF9D00FF9D00FF9D00FF9D00FF9D00B6
:10AE9000FF9D00FF9D00FF9D00FF9D00FF9D00FFA7
:10AEA0009D00FF9D00FF9D00FF9D00FF9D00FF9DF9
:10AEB00000FF9D00FF9D00FF9D00FF9D00FF9D0086
:10AEC000FF9D00FF9D00FF9D00FF9D00FF9D00FF77
:10AED0009D00FF9D00FF9D00FF9D00FF9D00FF9DC9
:10AEE00000FF9D00FF9D00FF9D00FF9D00FF9D0056
:10AEF000FF9D00FF9D00FF9D00FF9D00FF9D00FF47
:10AF00009D00FF9D00FF9D00FF9D00FF9D00FF9D98
:10AF100000FF9D00FF9D00FF9D00FF9D00FF9D0025
:10AF2000FF9D00FF9D00FF9D00FF9D00FF9D00FF16
:10AF30009D00FF9D00FF9D00FF9D00FF9D00FF9D68
:10AF400000FF9D00FF9D00FF9D00FF9D00FF9D00F5
:10AF5000FF9D00FF9D00FF9D00FF9D00FF9D00FFE6
:10AF60009D00FF9D00FF9D00FF9D00FF9D00FF9D38
:10AF700000FF9D00FF9D00FF9D00FF9D00FF9D00C5
:10AF8000FF9D00FF9D00000010212042306340849F
:10AF900050A560C670E781089129A14AB16BC18CA8
:10AFA000D1ADE1CEF1EF123102103273225252B51F
:10AFB000429472F762D693398318B37BA35AD3BDF8
:10AFC000C39CF3FFE3DE246234430420140164E6EF
:10AFD00074C744A45485A56AB54B85289509E5EE48
:10AFE000F5CFC5ACD58D365326721611063076D7FF
:10AFF00066F6569546B4B75BA77A97198738F7DF98
:10B00000E7FED79DC7BC48C458E5688678A70840C6
:10B01000186128023823C9CCD9EDE98EF9AF8948E7
:10B020009969A90AB92B5AF54AD47AB76A961A715E
:10B030000A503A332A12DBFDCBDCFBBFEB9E9B7937
:10B040008B58BB3BAB1A6CA67C874CE45CC52C22AE
:10B050003C030C601C41EDAEFD8FCDECDDCDAD2A87
:10B06000BD0B8D689D497E976EB65ED54EF43E133E
:10B070002E321E510E70FF9FEFBEDFDDCFFCBF1BD7
:10B08000AF3A9F598F78918881A9B1CAA1EBD10CB1
:10B09000C12DF14EE16F108000A130C220E35004B9
:10B0A00040257046606783B99398A3FBB3DAC33D2C
:10B0B000D31CE37FF35E02B1129022F332D2423509
:10B0C000521462777256B5EAA5CB95A88589F56EBC
:10B0D000E54FD52CC50D34E224C314A00481746659
:10B0E000644754244405A7DBB7FA879997B8E75F0C
:10B0F000F77EC71DD73C26D336F2069116B06657A9
:10B10000767646155634D94CC96DF90EE92F99C893
:10B1100089E9B98AA9AB584448657806682718C0F8
:10B1200008E1388228A3CB7DDB5CEB3FFB1E8BF96B
:10B130009BD8ABBBBB9A4A755A546A377A160AF148
:10B140001AD02AB33A92FD2EED0FDD6CCD4DBDAA7B
:10B15000AD8B9DE88DC97C266C075C644C453CA298
:10B160002C831CE00CC1EF1FFF3ECF5DDF7CAF9B4B
:10B17000BFBA8FD99FF86E177E364E555E742E93E8
:0CB180003EB20ED11EF0010000000000E5
:00000001FF
